:020000040000FA
:0400000027EF04F0F2
:080008005AEF10F0116A156AAD
:10001000146E010E0B6E1550115C02E11450105C51
:10002000040ED8B0010ED8B4020E0B14D8A4010EE1
:100030001200096A186E196A00960950D8B4008631
:10004000050E086E270E156E100E0CD8030E156ED9
:10005000E80E08D8156A640E05D8156A0A0E02D88B
:10006000185008D0146E1950116E1850106EB0EC64
:1000700001F01050106E084E0096095003E0085C25
:10008000D8B008D01050D8A4009600B603D0300FD6
:10009000D5EF00F01200356E21AE03D02D0ED5EC59
:1000A00000F0233E04D0223E02D0214A212A2A6AAF
:1000B0002B6A2C6A2D6A218E6A0E2026D890213256
:1000C000223223322D322C322B322A32203EF6D7E6
:1000D0002350205C2326205E2250215C2226215EB4
:1000E000096A3AD82E0ED5EC00F0366AD8902A3438
:1000F000236E2B34226E2C34216E2D34206E363636
:10010000D890233622362136203636362A502326FA
:100110002B50D8B02B3C22262C50D8B02C3C21267A
:100120002D50D8B02D3C2026D8B0363ED89023365E
:1001300022362136203636363650300FD5EC00F0D8
:1001400023C02AF022C02BF021C02CF020C02DF0BB
:10015000352ECBD7D89012000096095003E10086C7
:100160000A0E096E23C013F022C012F021C011F054
:1001700020C010F0086A1B6A1A6A196A0A0E186E03
:1001800053EC01F0082A0850095CD8A4F4D71850A1
:10019000D8A4009600A602D0092C04D01850300F25
:1001A000D5EC00F0092EDED7120001A205D001B077
:1001B00003D001B2EE6E1200A96EA66AA680A85006
:1001C000A92A1200A86EA66AA684550EA76EAA0ECA
:1001D000A76EA682A6B2FED7A694A92A1200E83678
:1001E000E8363C0B0109C212C009C216C050F80B18
:1001F0000309C06E320E48EC01F0C282C2B2FED7D3
:10020000C4CF21F0C350206E1200080E1C6E0F0EDA
:10021000EA6E06C0E9FF07500BB4D5EC01F00BA461
:10022000D7EC01F00F0EE26E06C0E1FF0F0EEA6E92
:1002300005C0E9FF0A1CE988E92AEC161C50D8B46D
:1002400012000BB0C7EC01F005C0E9FF113210320B
:10025000EF500A10D8A00A18EF6E03D81C2EF6D75C
:1002600012000750E71A000000D000D000D000D0E4
:1002700000D0E71A1200156A146EFF0E142615221C
:1002800000D0D8A01200030E116EE60E02D8F5D7EA
:10029000116AFC0F106E0000E86A01D01006000021
:1002A000115AFCE2120013501B18800BF46E13AEAF
:1002B00006D0D880000E10561156125613561BAE9B
:1002C00006D0D880000E185619561A561B56146AB6
:1002D000156A166A176A266A276A286A296A1B50ED
:1002E0001A101910181023E0200EF36ED890103653
:1002F0001136123613362636273628362936185048
:10030000265C195027581A5028581B50295809E3C1
:100310001850265E1950275A1A50285A1B50295A2D
:10032000D8801436153616361736F32EDFD7F4AECE
:1003300006D0D880000E145615561656175614C0FF
:1003400010F015C011F016C012F017C013F026C03F
:1003500018F027C019F028C01AF029C01BF01200AD
:10036000196A186A100EF36E1134183619361450C3
:10037000185C1550195805E31450185E1550195A99
:10038000D88010361136F32EEFD710501200146AB1
:10039000156A04D01132103214361536FF0FFAE206
:1003A00015C011F01450106E1200EF1203D0FF0AA6
:1003B000EF1601D0FF0AE988E92AEC1612002F5047
:1003C0002B18396E39BE30D02FBE17D02E502A5C74
:1003D000D8A0000CD8A4010C2F502B5CD8A0000C86
:1003E000D8A4010C30502C5CD8A0000CD8A4010C6F
:1003F00031502D5CD8A0000C010C2A502E5CD8A0E6
:10040000000CD8A4010C2B502F5CD8A0000CD8A451
:10041000010C2C50305CD8A0000CD8A4010C2D503D
:10042000315CD8A0000C010C2BAE010C000C2F503D
:100430002B18396E39BE34D02FBE19D02E502A5CFD
:10044000D8A0000CD8A4010C2F502B5CD8A0000C15
:10045000D8A4010C30502C5CD8A0000CD8A4010CFE
:1004600031502D5CD8A0000CD8A4010C000C2A50EF
:100470002E5CD8A0000CD8A4010C2B502F5CD8A067
:10048000000CD8A4010C2C50305CD8A0000CD8A4CF
:10049000010C2D50315CD8A0000CD8A4010C000C2C
:1004A0002BAE010C000C2B502F18396E39BE34D0F6
:1004B0002BBE19D02A502E5CD8A0000CD8A4010C59
:1004C0002B502F5CD8A0000CD8A4010C2C50305C11
:1004D000D8A0000CD8A4010C2D50315CD8A0000C81
:1004E000D8A4010C000C2E502A5CD8A0000CD8A473
:1004F000010C2F502B5CD8A0000CD8A4010C30505C
:100500002C5CD8A0000CD8A4010C31502D5CD8A0D4
:10051000000CD8A4010C000C2FAE010C000C800EB6
:100520002F1A2E502A5C366E11E2366C2A502EC0DD
:100530002AF02E6E2B502FC02BF02F6E2C5030C077
:100540002CF0306E2D5031C02DF0316E1A0E366009
:1005500078D02E5276E0356A2B50386E2F183A6ECE
:100560002B8E2F8E080E365E08E331C035F030C07A
:1005700031F02FC030F02F6AF5D7362607E0D8903B
:100580002F32303231323532362EF9D73AAE35D0BD
:1005900031502D5E30502C5A2F502B5A07E2D88004
:1005A000000E2D562C562B56800E381A356C04E052
:1005B0002D06000E2C5A2B5A040E366E2B660DD0CB
:1005C0002CC02BF02DC02CF035C02DF0356A080E54
:1005D0002A5E2DE3362EF2D72AD02BBE08D0D89033
:1005E00035362D362C362B362A2EF7D720D037AC81
:1005F00026D035AE24D0356A11D031502D2630505A
:100600002C222F502B2206E32B322C322D32353266
:100610002A4A0FD037AC13D035AE11D02D3E0FD0B3
:100620002C3E0DD02B3E0BD0D8802D90EDD72A6AD2
:1006300002D037822A682D6A2C6A800E2B6E38AE63
:100640002B9E2D5012002B50286E2F183A6E2E50D4
:1006500053E02A5254E02A5E7F0E03E22A2603E288
:100660004DD02A264EE22DC026F02CC027F0288E31
:100670002F8E180E386E2D6A2C6A2B6A0BD03150D3
:10068000265C3050275811E3276E286A3150265EC9
:100690000BD004E22F50285CF2E007E33150265ED5
:1006A0003050275A2F50285AD8802D362C362B36CA
:1006B000263627362836382EECD72BBE07D02A52BE
:1006C0001DE03A322A06382A3A36E3D737AC1FD033
:1006D00007E23150265E3050275A2F50285A17E330
:1006E0002D3E15D02C3E13D02B3E11D02B322C3268
:1006F0002D322A3E0CD005D0378604D037842A6AA2
:1007000002D037822A682D6A2C6A800E2B6E3AAE90
:100710002B9E2D5012002B50286E2F183A6E2A5007
:10072000D8A42E503CE02A267E0E03E32A5E03E383
:1007300038D02A5E33E32DC026F02CC027F0288E57
:100740002F8E2D6A2C6A2B6A180E386E28322732AB
:10075000263206E331502D2630502C222F502B22EA
:100760002B322C322D32382EF1D72BBE07D02D361E
:100770002C362B362A5212E02A06283437AC17D0F2
:1007800016E32D3E14D02C3E12D02B3E10D0D88034
:100790002B322C322D322A3E0AD003D037842A6ADB
:1007A00002D037822A682D6A2C6A800E2B6E3AAEF0
:1007B0002B9E2D5012002C6A2D6A960E386E3A9E92
:1007C0002DAE07D0D880000E2A562B562C562D560B
:1007D0003A8E2D5218E037AC0DD02DAE0BD02B2A0F
:1007E00009E12C2A07E12D2A05E1D8802D322C328F
:1007F0002B32382A080E38262BC02AF02CC02BF0BA
:100800002DC02CF011D02C520FE1080E385E2B5069
:1008100007E1080E385E2A5002E12D5010D02A6AF6
:100820002C6E2AC02BF02A6A2CBE06D0D8902A360D
:100830002B362C363806F8D73AAE2C9E38502AC0C4
:100840002DF02A6E2C502BC02CF02B6E1200F86A63
:10085000400E376E006AAB6A0001B468C16AF19E4F
:10086000010E156EF40E3CEC01F0E80E3B6E030E2B
:100870003C6EF40E3D6E010E3E6E810E946EF20ED5
:10088000936EE80EC26EFC0EC16E050EB46ECF0EF6
:10089000926E819681908292C08E696A686A676A58
:1008A000666A716A706A6F6A6E6ADB0EBF6F0F0EDE
:1008B000BE6F490EBD6F800EBC6F01010A6B096BE4
:1008C000086B076B640EDCEC00F00B6F640E0B5DC5
:1008D000010ED8B0E86A326E0BC110F0FA0E06ECC9
:1008E00000F032120001D8B47EEF04F0BF0E010117
:1008F0000B6F0001B7EC23F062EF19F050EC18F029
:10090000B7EC23F0010EDCEC00F09B6FDDEC00F0A7
:100910009C6FDDEC00F09D6FDDEC00F09E6F63ECF2
:100920001EF0D8969CBFD886D8B6B6EF04F0010E5C
:100930009E5D800E9D593B0E9C59890E9B59D8A0F7
:10094000B6EF04F09E6B9D6B7A0E9C6F880E9B6FCA
:10095000010EA96E9B51E2EC00F09C51E2EC00F01C
:100960009D51E2EC00F09E51E2EC00F09CBF0BD0F8
:10097000000E9E5D000E9D597A0E9C59870E9B5964
:10098000D8B0D7EF04F09E6B9D6B7A0E9C6F880EEB
:100990009B6F010EA96E9B51E2EC00F09C51E2ECC2
:1009A00000F09D51E2EC00F09E51E2EC00F00A0EE6
:1009B000DCEC00F0C881E8A0C8910B0EDCEC00F084
:1009C000C883E8A0C8930C0EDCEC00F0C46FDDEC2B
:1009D00000F0C56FDDEC00F0C66FDDEC00F0C76F16
:1009E000C7BF0CD0C651C711D8A400EF05F04D0EFB
:1009F000C45D040EC559D8B000EF05F0000E01D05B
:100A0000010E326ED896C7BFD886D8B621EF05F052
:100A1000000EC75DD8A021EF05F011E1000EC65D04
:100A2000D8A021EF05F00BE1030EC55DD8A021EFA2
:100A300005F005E1840EC45DD8A021EF05F0000E9D
:100A400001D0010E3212D8B42CEF05F0C76BC66B83
:100A5000030EC56FE80EC46FC831E832D8A032EF7C
:100A600005F08180C831E832D8B038EF05F08190C8
:100A7000640E3BEC01F072EC26F0070E156ED00E02
:100A80003CEC01F019EC16F07FEC24F07AEC2CF041
:100A9000AAEC2EF022EC2FF0A5EF0CF07AEC2CF063
:100AA000AAEC2EF0436A010E446E97EC24F0200E5F
:100AB0004D6E4E6E4F6E506E516E526E536E546E42
:100AC000556E566E576E586E596E5A6E5B6A61EC73
:100AD00024F0436A020E446E97EC24F0200E4D6E13
:100AE0004E6E4F6E506E516E526E536E546E556E0A
:100AF000566E576E586E596E5A6E5B6A61EC24F0F2
:100B0000436A030E446E97EC24F0200E4D6E4E6E39
:100B10004F6E506E516E526E536E546E556E566ED1
:100B2000576E586E596E5A6E5B6A61EC24F03EC087
:100B300015F03D503CEC01F019EC16F08FEC08F08C
:100B400082AEAEEF05F030EC22F05FEC0DF06AEC17
:100B50000DF0BDEC05F0F8EC08F0EED782BEBCEF6E
:100B600005F084EC22F05FEC0DF063EC0EF075EC18
:100B700007F0F8EC08F0E0D7DFD7D896A0BFD8860A
:100B8000D8B6C8EF05F07F0E9F5DD8B0CCEF05F06A
:100B9000A26BA16BA06B9F6BA0BF0BD0000EA25DE0
:100BA000000EA1597A0EA059880E9F59D8B0F6EFC1
:100BB00005F0030E436E020E446E97EC24F0200EF7
:100BC0004D6E4E6E4F6E506E516E526E536E546E31
:100BD000556E566E700E576E460E586E200E596E3C
:100BE0005A6E5B6A61EC24F014EF07F0A2C02DF09E
:100BF000A1C02CF0A0C02BF09FC02AF0316A306A4F
:100C00007A0E2F6E880E2E6EDFEC01F0326EA2C0CF
:100C10002DF0A1C02CF0A0C02BF09FC02AF0316AAB
:100C2000500E306E430E2F6E8F0E2E6E53EC02F070
:100C30003216D8B451EF06F0316A306A7A0E2F6E50
:100C4000880E2E6EA2C02DF0A1C02CF0A0C02BF0FB
:100C50009FC02AF023EC03F02DC0A2F02CC0A1F01D
:100C60002BC0A0F02AC09FF0030E436E020E446E0C
:100C700097EC24F0200E4D6E4E6E4F6E506E516EFE
:100C8000526E536E546E556E566E6E0E576E460E05
:100C9000586E200E596E5A6E5B6A61EC24F02DEF8F
:100CA00007F0A2C02DF0A1C02CF0A0C02BF09FC077
:100CB0002AF0316A500E306E430E2F6E8F0E2E6E5C
:100CC000DFEC01F0326EA2C02DF0A1C02CF0A0C06C
:100CD0002BF09FC02AF0316A240E306E740E2F6EF6
:100CE000920E2E6E53EC02F03216D8B4AEEF06F030
:100CF000316A240E306E740E2F6E920E2E6EA2C0CC
:100D00002DF0A1C02CF0A0C02BF09FC02AF023EC46
:100D100003F02DC0A2F02CC0A1F02BC0A0F02AC07F
:100D20009FF0030E436E020E446E97EC24F0200EEB
:100D30004D6E4E6E4F6E506E516E526E536E546EBF
:100D4000556E566E750E576E460E586E200E596EC5
:100D50005A6E5B6A61EC24F045EF07F02D6A500E85
:100D60002C6E430E2B6E8F0E2A6EA2C031F0A1C0E6
:100D700030F0A0C02FF09FC02EF017EC02F0010859
:100D8000D8B4F9EF06F0316A240E306E740E2F6E6F
:100D9000920E2E6EA2C02DF0A1C02CF0A0C02BF0A0
:100DA0009FC02AF023EC03F02DC0A2F02CC0A1F0CC
:100DB0002BC0A0F02AC09FF0030E436E020E446EBB
:100DC00097EC24F0200E4D6E4E6E4F6E506E516EAD
:100DD000526E536E546E556E566E750E576E460EAD
:100DE000586E200E596E5A6E5B6A61EC24F05DEF0E
:100DF00007F0030E436E020E446E97EC24F0200EB3
:100E00004D6E4E6E4F6E506E516E526E536E546EEE
:100E1000556E566E700E576E460E586E200E596EF9
:100E20005A6E5B6A61EC24F0140E436E020E446E3F
:100E300097EC24F000EE4DF0020E016EA2C023F0FC
:100E4000A1C022F0A0C021F09FC020F0010E4BEC09
:100E500000F0EF6A61EC24F01200140E436E020EF3
:100E6000446E97EC24F000EE4DF0020E016EA2C02D
:100E700023F0A1C022F0A0C021F09FC020F04BECD5
:100E800000F0EF6A61EC24F01200140E436E020EC3
:100E9000446E97EC24F000EE4DF0020E016EA2C0FD
:100EA00023F0A1C022F0A0C021F09FC020F04BECA5
:100EB00000F0EF6A61EC24F01200140E436E020E93
:100EC000446E97EC24F000EE4DF0020E016EA2C0CD
:100ED00023F0A1C022F0A0C021F09FC020F04BEC75
:100EE00000F0EF6A61EC24F01200A4BF0BD0CD0E2D
:100EF000A65DCC0EA5594C0EA4597B0EA359D8B0B3
:100F0000B7EF07F02D6A2C6A7A0E2B6E880E2A6EC8
:100F1000A6C031F0A5C030F0A4C02FF0A3C02EF0C1
:100F20008BEC03F02DC0A6F02CC0A5F02BC0A4F0D4
:100F30002AC0A3F0030E436E020E446E97EC24F019
:100F4000200E4D6E4E6E4F6E506E516E526E536E41
:100F5000546E556E6E0E566E480E576E200E586EBD
:100F6000596E5A6E5B6A61EC24F045EF08F0A6C03A
:100F70002DF0A5C02CF0A4C02BF0A3C02AF0CD0EFC
:100F8000316ECC0E306E4C0E2F6E7B0E2E6EDFEC63
:100F900001F0326EA6C02DF0A5C02CF0A4C02BF03D
:100FA000A3C02AF0316A306A2F6A7F0E2E6E53EC8E
:100FB00002F03216D8B4FAEF07F0030E436E020EB9
:100FC000446E97EC24F0200E4D6E4E6E4F6E506EB8
:100FD000516E526E536E546E556E750E566E480EAF
:100FE000576E200E586E596E5A6E5B6A61EC24F093
:100FF0005EEF08F02D6A2C6A2B6A7F0E2A6EA6C05F
:1010000031F0A5C030F0A4C02FF0A3C02EF017EC33
:1010100002F00108D8B42AEF08F0030E436E020E66
:10102000446E97EC24F0200E4D6E4E6E4F6E506E57
:10103000516E526E536E546E556E750E566E480E4E
:10104000576E200E586E596E5A6E5B6A61EC24F032
:1010500076EF08F0030E436E020E446E97EC24F018
:10106000200E4D6E4E6E4F6E506E516E526E536E20
:10107000546E556E6E0E566E480E576E200E586E9C
:10108000596E5A6E5B6A61EC24F0190E436E020EC3
:10109000446E97EC24F000EE4DF0020E016EA6C0F7
:1010A00023F0A5C022F0A4C021F0A3C020F0010EBF
:1010B0004BEC00F0EF6A61EC24F01200190E436E65
:1010C000020E446E97EC24F000EE4DF0020E016E1D
:1010D000A6C023F0A5C022F0A4C021F0A3C020F038
:1010E0004BEC00F0EF6A61EC24F01200190E436E35
:1010F000020E446E97EC24F000EE4DF0020E016EED
:10110000A6C023F0A5C022F0A4C021F0A3C020F007
:10111000010E4BEC00F0EF6A61EC24F0120081BE8E
:1011200096EF08F05EEC23F0F8EF10F081BC9DEF35
:1011300008F05EEC23F0B9EF1DF081B8A4EF08F0E1
:10114000DEEC22F0A5EF0CF081BAADEF08F05EEC1A
:1011500023F033EC1CF0AEEC08F012007AEC2CF02B
:10116000AAEC2EF0436A010E446E97EC24F0200E98
:101170004D6E4E6E4F6E506E516E526E536E546E7B
:10118000556E566E576E586E596E5A6E5B6A61ECAC
:1011900024F0436A020E446E97EC24F0200E4D6E4C
:1011A0004E6E4F6E506E516E526E536E546E556E43
:1011B000566E576E586E596E5A6E5B6A61EC24F02B
:1011C000436A030E446E97EC24F0200E4D6E4E6E73
:1011D0004F6E506E516E526E536E546E556E566E0B
:1011E000576E586E596E5A6E5B6A61EC24F01200AD
:1011F00097518F5DC96F98519059CA6F9951915904
:10120000CB6F9A519259CC6F436A040E446E97EC9F
:1012100024F094988288456A466A4652D8A41EEF04
:101220000BF0540E455CD8B01EEF0BF0D896CCBF37
:10123000D886D8B646EF09F0000ECC5DD8A046EFB0
:1012400009F011E1000ECB5DD8A046EF09F00BE1EB
:10125000000ECA5DD8A046EF09F005E1280EC95D71
:10126000D8A046EF09F0170E0F6E9C0E0E6E45507B
:101270000E24F66E46500F20F76EA66AA68E080062
:10128000F5CF0CF00CC04DF00AEF0BF0CCBF11D035
:10129000CC53D8A45BEF09F0CB53D8A45BEF09F093
:1012A000CA53D8A45BEF09F0C9511D08D8A05BEF61
:1012B00009F0000E01D0010E326ED896CCBFD88650
:1012C000D8B66EEF09F0CA51CB11CC1105E1280E4A
:1012D000C95DD8A06EEF09F0000E01D0010E3216E4
:1012E000D8B486EF09F0170E0F6E460E0E6E4550FD
:1012F0000E24F66E46500F20F76EA66AA68E0800E2
:10130000F5CF0CF00CC04DF00AEF0BF0CCBF11D0B4
:10131000CC53D8A49BEF09F0CB53D8A49BEF09F092
:10132000CA53D8A49BEF09F0C9511308D8A09BEF6A
:1013300009F0000E01D0010E326ED896CCBFD886CF
:10134000D8B6AEEF09F0CA51CB11CC1105E11E0E93
:10135000C95DD8A0AEEF09F0000E01D0010E321623
:10136000D8B4C6EF09F0160E0F6EF00E0E6E455093
:101370000E24F66E46500F20F76EA66AA68E080061
:10138000F5CF0CF00CC04DF00AEF0BF0CCBF11D034
:10139000CC53D8A4DBEF09F0CB53D8A4DBEF09F092
:1013A000CA53D8A4DBEF09F0C9510908D8A0DBEF74
:1013B00009F0000E01D0010E326ED896CCBFD8864F
:1013C000D8B6EEEF09F0CA51CB11CC1105E1140EDD
:1013D000C95DD8A0EEEF09F0000E01D0010E321663
:1013E000D8B406EF0AF0160E0F6E9A0E0E6E455028
:1013F0000E24F66E46500F20F76EA66AA68E0800E1
:10140000F5CF0CF00CC04DF00AEF0BF0D896CCAF36
:10141000D886D8B60EEF0AF0000E01D0010E326E5B
:10142000D896CCBFD886D8B621EF0AF0CA51CB11D6
:10143000CC1105E10A0EC95DD8A021EF0AF0000E1B
:1014400001D0010E3216D8B439EF0AF0160E0F6E25
:10145000440E0E6E45500E24F66E46500F20F76E69
:10146000A66AA68E0800F5CF0CF00CC04DF00AEF6E
:101470000BF0D896CCBFD886D8B641EF0AF0000E54
:1014800001D0010E326ED896CCAFD886D8B656EFC2
:101490000AF0F60EC95DFF0ECA59FF0ECB59FF0EBA
:1014A000CC59D8B056EF0AF0000E01D0010E32161A
:1014B000D8B46EEF0AF0170E0F6EF20E0E6E455096
:1014C0000E24F66E46500F20F76EA66AA68E080010
:1014D000F5CF0CF00CC04DF00AEF0BF0CCAF0BD0F9
:1014E000F60EC95DFF0ECA59FF0ECB59FF0ECC593F
:1014F000D8A07DEF0AF0000E01D0010E326ED89612
:10150000CCAFD886D8B692EF0AF0EC0EC95DFF0ECC
:10151000CA59FF0ECB59FF0ECC59D8B092EF0AF042
:10152000000E01D0010E3216D8B4AAEF0AF0180E40
:101530000F6E480E0E6E45500E24F66E46500F206C
:10154000F76EA66AA68E0800F5CF0CF00CC04DF021
:101550000AEF0BF0CCAF0BD0EC0EC95DFF0ECA59F1
:10156000FF0ECB59FF0ECC59D8A0B9EF0AF0000EF0
:1015700001D0010E326ED896CCAFD886D8B6CEEF59
:101580000AF0E20EC95DFF0ECA59FF0ECB59FF0EDD
:10159000CC59D8B0CEEF0AF0000E01D0010E3216B1
:1015A000D8B4E6EF0AF0180E0F6E9E0E0E6E455080
:1015B0000E24F66E46500F20F76EA66AA68E08001F
:1015C000F5CF0CF00CC04DF00AEF0BF0D896CCAF75
:1015D000D886D8B60AEF0BF0E20EC95DFF0ECA59E5
:1015E000FF0ECB59FF0ECC59D8B00AEF0BF0180EF6
:1015F0000F6EF40E0E6E45500E24F66E46500F2000
:10160000F76EA66AA68E0800F5CF0CF00CC04DF060
:101610000AEF0BF0820E056E080E0A6E820E066E41
:10162000040E076E010E0B6E4D50106E05EC01F0AE
:10163000452AD8B4462AD8A40DEF09F0640E48EC28
:1016400001F01200809CA28888888888A29C8080F3
:1016500080888888889C88888888889C88888888EA
:10166000889C88888888889C888888889CBEBE9C3E
:10167000888888889C88888888889C8888888888C2
:101680009C88888888889C888888888080809CA29C
:101690008888BE8888A29C801200809CA288888846
:1016A0008888A29C808080888888889C8888888890
:1016B000889C88888888889C88888888889C88886E
:1016C0008888889C9C888888889CBE9C8888888814
:1016D0009C88888888889C88888888889C8888884E
:1016E000888080809CA28888BE8888A29C80120006
:1016F000809CA28888888888A29C8080808888882E
:10170000889C88888888889C88888888889C88881D
:101710008888889C88888888889C9C88888888880D
:101720009C888888889CBE9C888888889C888888B3
:1017300088889C888888888080809CA28888BE88C9
:1017400088A29C801200809CA28888888888A29C9D
:10175000808080888888889C88888888889C8888F9
:101760008888889C88888888889C88888888889CBD
:101770009C88888888889C88888888889C888888AD
:10178000889CBE9C888888889C888888888080807F
:101790009CA28888BE8888A29C801200809CA28817
:1017A00088888888A29C808080888888889C88888F
:1017B0008888889C88888888889C88888888889C6D
:1017C00088888888889C9C88888888889C8888885D
:1017D00088889C88888888889C888888889CBE9C03
:1017E0008888888080809CA28888BE8888A29C8007
:1017F0001200809CA28888888888A29C808080882B
:101800008888889C88888888889C88888888889C1C
:10181000888888889CBE9C888888889C9C888888C2
:1018200088889C88888888889C88888888889C88FC
:10183000888888889C888888888080809CA28888FE
:10184000BE8888A29C801200809CA2888888888894
:10185000A29C808080888888889C88888888889CCA
:10186000888888889CBE9C888888889C8888888886
:10187000889C9C88888888889C88888888889C8898
:10188000888888889C88888888889C8888888880B8
:1018900080809CA28888BE8888A29C801200809C40
:1018A000A28888888888A29C808080888888889C74
:1018B000888888889CBE9C888888889C8888888836
:1018C000889C88888888889C9C88888888889C8848
:1018D000888888889C88888888889C888888888860
:1018E0009C888888888080809CA28888BE8888A2FE
:1018F0009C801200809CA28888888888A29C808016
:10190000808888889CBE9C888888889C88888888ED
:10191000889C88888888889C88888888889C9C88F7
:10192000888888889C88888888889C88888888880F
:101930009C88888888889C888888888080809CA2E9
:101940008888BE8888A29C80120022EC2FF0C0EC10
:101950002FF03EEC10F07AC092F079C091F078C090
:1019600090F077C08FF07AC07EF079C07DF078C0BB
:101970007CF077C07BF03EEC10F07AC082F079C04A
:1019800081F078C080F077C07FF03EEC10F07AC034
:1019900086F079C085F078C084F077C083F07F50FE
:1019A0007B24206E80517C20216E81517D20226E0F
:1019B00082517E20236E835120248F6F84512120F9
:1019C000906F85512220916F86512320926F92C093
:1019D00013F091C012F090C011F08FC010F01B6A8C
:1019E0001A6A196A030E186E53EC01F013C092F0D4
:1019F00012C091F011C090F010C08FF0828246ECBE
:101A00002FF03EEC10F07AC096F079C095F078C0D7
:101A100094F077C093F07AC07EF079C07DF078C002
:101A20007CF077C07BF03EEC10F07AC082F079C099
:101A300081F078C080F077C07FF03EEC10F07AC083
:101A400086F079C085F078C084F077C083F07F504D
:101A50007B24206E80517C20216E81517D20226E5E
:101A600082517E20236E83512024936F8451212044
:101A7000946F85512220956F86512320966F96C0D2
:101A800013F095C012F094C011F093C010F01B6ACF
:101A90001A6A196A030E186E53EC01F013C096F01F
:101AA00012C095F011C094F010C093F08292CC6BEC
:101AB000CB6BCA6BC96B04EC09F04EEF05F03EEC42
:101AC00010F07AC09AF079C099F078C098F077C099
:101AD00097F012009AC02DF099C02CF098C02BF00E
:101AE00097C02AF0DDEC03F02DC031F02CC030F0AF
:101AF0002BC02FF02AC02EF092C02DF091C02CF0F8
:101B000090C02BF08FC02AF0DDEC03F023EC03F043
:101B10002DC0ABF02CC0AAF02BC0A9F02AC0A8F0B1
:101B2000ABC031F0AAC030F0A9C02FF0A8C02EF091
:101B3000ABC02DF0AAC02CF0A9C02BF0A8C02AF091
:101B40008BEC03F02DC0ABF02CC0AAF02BC0A9F099
:101B50002AC0A8F0316A306A2F6A7F0E2E6EABC0A1
:101B60002DF0AAC02CF0A9C02BF0A8C02AF08FEC51
:101B700002F02DC0ABF02CC0AAF02BC0A9F02AC0F7
:101B8000A8F096C02DF095C02CF094C02BF093C017
:101B90002AF0DDEC03F02DC031F02CC030F02BC06A
:101BA0002FF02AC02EF092C02DF091C02CF090C0E2
:101BB0002BF08FC02AF0DDEC03F023EC03F02DC0F6
:101BC000AFF02CC0AEF02BC0ADF02AC0ACF0AFC06F
:101BD00031F0AEC030F0ADC02FF0ACC02EF0AFC0D1
:101BE0002DF0AEC02CF0ADC02BF0ACC02AF08BECC9
:101BF00003F02DC0AFF02CC0AEF02BC0ADF02AC06A
:101C0000ACF0316A306A2F6A7F0E2E6EAFC02DF0B5
:101C1000AEC02CF0ADC02BF0ACC02AF08FEC02F0BF
:101C20002DC0AFF02CC0AEF02BC0ADF02AC0ACF090
:101C3000ABC02DF0AAC02CF0A9C02BF0A8C02AF090
:101C4000AFC031F0AEC030F0ADC02FF0ACC02EF060
:101C500023EC03F02DC0A2F02CC0A1F02BC0A0F00B
:101C60002AC09FF0A2C031F0A1C030F0A0C02FF078
:101C70009FC02EF09EC02DF09DC02CF09CC02BF07C
:101C80009BC02AF08BEC03F02DC0A2F02CC0A1F079
:101C90002BC0A0F02AC09FF09F53D8B45AEF0EF08B
:101CA000D896A0AFD886D8B65AEF0EF0A26BA16B2B
:101CB000A06B9F6BA2C0F9F0A1C0F8F0A0C0F7F034
:101CC0009FC0F6F012009AC02DF099C02CF098C079
:101CD0002BF097C02AF0DDEC03F02DC031F02CC0C2
:101CE00030F02BC02FF02AC02EF092C02DF091C002
:101CF0002CF090C02BF08FC02AF0DDEC03F023EC29
:101D000003F02DC0ABF02CC0AAF02BC0A9F02AC064
:101D1000A8F0ABC031F0AAC030F0A9C02FF0A8C025
:101D20002EF0ABC02DF0AAC02CF0A9C02BF0A8C09B
:101D30002AF08BEC03F02DC023F02CC022F02BC036
:101D400021F02AC020F0316A306A2F6A7F0E2E6E91
:101D500023C02DF022C02CF021C02BF020C02AF08F
:101D60008FEC02F02DC0ABF02CC0AAF02BC0A9F074
:101D70002AC0A8F02D6A240E2C6E740E2B6E920EC3
:101D80002A6EABC031F0AAC030F0A9C02FF0A8C0B5
:101D90002EF08BEC03F02DC0ABF02CC0AAF02BC0C2
:101DA000A9F02AC0A8F096C02DF095C02CF094C0E0
:101DB0002BF093C02AF0DDEC03F02DC031F02CC0E5
:101DC00030F02BC02FF02AC02EF092C02DF091C021
:101DD0002CF090C02BF08FC02AF0DDEC03F023EC48
:101DE00003F02DC0AFF02CC0AEF02BC0ADF02AC078
:101DF000ACF0AFC031F0AEC030F0ADC02FF0ACC031
:101E00002EF0AFC02DF0AEC02CF0ADC02BF0ACC0AA
:101E10002AF08BEC03F02DC023F02CC022F02BC055
:101E200021F02AC020F0316A306A2F6A7F0E2E6EB0
:101E300023C02DF022C02CF021C02BF020C02AF0AE
:101E40008FEC02F02DC0AFF02CC0AEF02BC0ADF087
:101E50002AC0ACF02D6A2C6A7A0E2B6E880E2A6E80
:101E6000AFC031F0AEC030F0ADC02FF0ACC02EF03E
:101E70008BEC03F02DC0AFF02CC0AEF02BC0ADF05A
:101E80002AC0ACF02D6A2C6A7A0E2B6E880E2A6E50
:101E90009EC031F09DC030F09CC02FF09BC02EF052
:101EA00023EC03F02DC0B3F02CC0B2F02BC0B1F086
:101EB0002AC0B0F092C02DF091C02CF090C02BF051
:101EC0008FC02AF0DDEC03F0560E316E0E0E306E30
:101ED000490E2F6E810E2E6E8BEC03F02DC0B7F0E5
:101EE0002CC0B6F02BC0B5F02AC0B4F02D6A240E79
:101EF0002C6E740E2B6E920E2A6EB7C031F0B6C0E7
:101F000030F0B5C02FF0B4C02EF023EC03F02DC09C
:101F1000B7F02CC0B6F02BC0B5F02AC0B4F0B7C0F3
:101F200031F0B6C030F0B5C02FF0B4C02EF0B7C05D
:101F30002DF0B6C02CF0B5C02BF0B4C02AF08BEC5D
:101F400003F02DC0B7F02CC0B6F02BC0B5F02AC0FE
:101F5000B4F0ABC031F0AAC030F0A9C02FF0A8C0D7
:101F60002EF0B7C02DF0B6C02CF0B5C02BF0B4C029
:101F70002AF08BEC03F02DC0BBF02CC0BAF02BC0C4
:101F8000B9F02AC0B8F0316A306A7A0E2F6E880E26
:101F90002E6EBBC02DF0BAC02CF0B9C02BF0B8C06B
:101FA0002AF023EC03F02DC0BBF02CC0BAF02BC0FC
:101FB000B9F02AC0B8F0B3C031F0B2C030F0B1C04F
:101FC0002FF0B0C02EF0AFC02DF0AEC02CF0ADC0E1
:101FD0002BF0ACC02AF08BEC03F02DC023F12CC009
:101FE00022F12BC021F12AC020F123C131F022C1FE
:101FF00030F021C12FF020C12EF0BBC02DF0BAC0AF
:102000002CF0B9C02BF0B8C02AF08BEC03F02DC037
:10201000A6F02CC0A5F02BC0A4F02AC0A3F0316A12
:10202000306A7A0E2F6E880E2E6EA6C02DF0A5C0D7
:102030002CF0A4C02BF0A3C02AF023EC03F02DC099
:10204000A6F02CC0A5F02BC0A4F02AC0A3F0A35387
:10205000D8B435EF10F0D896A4AFD886D8B635EFFF
:1020600010F0A66BA56BA46BA36BA6C0F9F0A5C07E
:10207000F8F0A4C0F7F0A3C0F6F012000101256B40
:10208000020ECD6E9E90CF6ACE6A9D80F29E070EA4
:10209000D56EF294D90ED76EDA0ED66EF28AF28E23
:1020A000F28CD58ECD800001F2A459EF10F074EFC0
:1020B00010F0F9D7F2A45FEF10F074EF10F0F29E79
:1020C000020ECD6E9E90CF6ACE6A9D80F28ECD803C
:1020D0000101252B03C0E9FF04C0EAFF02C0E0FFB5
:1020E000345033C0D8FF10000001F29ED59ECD9031
:1020F0000600766A756A746A736ACECF26F1CFCF0E
:1021000027F126C173F027C174F0756A766A010E53
:102110000101255D0001D8A495EF10F0000E732693
:102120007422010E7522000E7622020E0101255D39
:102130000001D8A4A3EF10F0000E73267422020E43
:102140007522000E7622030E0101255D0001D8A440
:10215000B1EF10F0000E73267422030E7522000EEC
:102160007622040E0101255D0001D8A4BFEF10F016
:10217000000E73267422040E7522000E7622050EC0
:102180000101255D0001D8A4CDEF10F0000E7326EB
:102190007422050E7522000E7622060E0101255DC1
:1021A0000001D8A4DBEF10F0000E73267422060E97
:1021B0007522000E762276C07AF075C079F074C070
:1021C00078F073C077F0E80E775E030E785A000E51
:1021D000795A7A5AC4517726C5517822C651792244
:1021E000C7517A22D8907736783679367A36120007
:1021F0007FEC24F006EC2DF0E6EC2EF0436A446A06
:1022000097EC24F0200E4D6E4E6E4F6E506E530EB6
:10221000516E650E526E740E536E750E546E700EC6
:10222000556E200E566E576E586E596E5A6E5B6A1A
:1022300061EC24F03EC015F03D503CEC01F0010E85
:10224000726E4CEC11F081BC30EF11F05EEC23F0BB
:10225000722A4CEC11F03EC015F03D503CEC01F000
:1022600081B83DEF11F05EEC23F072064CEC11F0FA
:102270003EC015F03D503CEC01F081BE44EF11F042
:102280005EEC23F04EEF05F081BA4BEF11F05EECFF
:1022900023F0B4EF11F0D7D77252D8A452EF11F057
:1022A000090E726E0A0E725CD8A459EF11F0010E7D
:1022B000726E010E725CD8A463EF11F0F3EC11F0B2
:1022C000656A0EEC12F0020E725CD8A46DEF11F08C
:1022D000F3EC11F0656A2EEC12F0030E725CD8A4D8
:1022E00077EF11F0F3EC11F0656A4DEC12F0040E8B
:1022F000725CD8A481EF11F0FCEC11F0656A6CEC13
:1023000012F0050E725CD8A48BEF11F0FCEC11F00A
:10231000656A8FEC12F0060E725CD8A495EF11F08E
:10232000FCEC11F0656AB2EC12F0070E725CD8A4F6
:102330009FEF11F005EC12F0656AD4EC12F0080E74
:10234000725CD8A4A9EF11F005EC12F0656AF4EC08
:1023500012F0090E725CD8A4B3EF11F005EC12F084
:10236000656A13EC13F01200010E725CD8A4BBEF87
:1023700011F0F5EF1FF0020E725CD8A4C2EF11F05D
:10238000A3EF1BF0030E725CD8A4C9EF11F0ECEFC1
:102390001BF0040E725CD8A4D0EF11F05FEF1CF0BC
:1023A000050E725CD8A4D7EF11F0B1EF1AF0060E4B
:1023B000725CD8A4DEEF11F062EF19F0070E725CC8
:1023C000D8A4E5EF11F088EF13F0080E725CD8A4E2
:1023D000ECEF11F05EEF1DF0090E725CD8A4F3EF84
:1023E00011F05EEF1DF0010E656E0EEC12F02EEC9A
:1023F00012F04DEC12F01200010E656E6CEC12F052
:102400008FEC12F0B2EC12F01200010E656ED4ECFB
:1024100012F0F4EC12F013EC13F01200436A010E08
:10242000446E97EC24F0310E4D6E2E0E4E6E4D0E16
:102430004F6E650E506E6D0E516E6F0E526E720EB7
:10244000536E790E546E200E556E566E576E586E42
:10245000596E5A6E5B6A61EC24F01200436A020EF8
:10246000446E97EC24F0320E4D6E2E0E4E6E530ECF
:102470004F6E6F0E506E750E516E6E0E526E640E74
:10248000536E200E546E556E566E576E586E596EC2
:102490005A6E5B6A61EC24F01200436A030E446ECC
:1024A00097EC24F0330E4D6E2E0E4E6E4C0E4F6E8A
:1024B000690E506E670E516E680E526E740E536E3A
:1024C000200E546E556E566E576E586E596E5A6E7B
:1024D0005B6A61EC24F01200436A010E446E97ECD3
:1024E00024F0340E4D6E2E0E4E6E4F0E4F6E730E48
:1024F000506E630E516E690E526E6C0E536E546EBA
:10250000610E556E740E566E6F0E576E720E586ECB
:10251000200E596E5A6E5B6A61EC24F01200436A19
:10252000020E446E97EC24F0350E4D6E2E0E4E6E5C
:10253000430E4F6E610E506E700E516E610E526EF4
:10254000630E536E690E546E740E556E6F0E566E9A
:10255000720E576E200E586E596E5A6E5B6A61ECA1
:1025600024F01200436A030E446E97EC24F0360EFA
:102570004D6E2E0E4E6E430E4F6E6F0E506E6E0EE3
:10258000516E740E526E720E536E610E546E730E57
:10259000556E740E566E200E576E586E596E5A6EEA
:1025A0005B6A61EC24F01200436A010E446E97EC02
:1025B00024F0370E4D6E2E0E4E6E420E4F6E610E93
:1025C000506E740E516E526E650E536E720E546ED6
:1025D000790E556E200E566E576E586E596E5A6EA5
:1025E0005B6A61EC24F01200436A020E446E97ECC1
:1025F00024F0380E4D6E2E0E4E6E410E4F6E620E52
:10260000506E6F0E516E750E526E740E536E200E1C
:10261000546E556E566E576E586E596E5A6E5B6A92
:1026200061EC24F01200436A030E446E97EC24F030
:10263000760E4D6E2E0E4E6E200E4F6E320E506E7A
:10264000516E2E0E526E300E536E350E546E2E0E8F
:10265000556E320E566E300E576E310E586E300E6D
:10266000596E200E5A6E5B6A61EC24F01200190E4E
:10267000436E446A97EC24F094988288456A466ACF
:102680004652D8A46DEF13F0300E455CD8B06DEF14
:1026900013F0260E0F6EDC0E0E6E45500E24F66EF5
:1026A00046500F20F76EA66AA68E0800F5CF0CF0F4
:1026B0000CC04DF0820E056E080E0A6E820E066E7C
:1026C000040E076E010E0B6E4D50106E05EC01F0FE
:1026D000452AD8B4462AD8A4D3D71200006F494956
:1026E000497B78007C54545C00047F74007C70400B
:1026F0007C007E72121E000000000000000000003E
:1027000000000000000000000000000000001200B7
:10271000010E726E7FEC24F006EC2DF03EC015F039
:102720003D503CEC01F0BEEC13F081BCA2EF13F085
:102730005EEC23F0722ABEEC13F03EC015F03D5063
:102740003CEC01F081B8AFEF13F05EEC23F07206C1
:10275000BEEC13F03EC015F03D503CEC01F081BEE4
:10276000B6EF13F05EEC23F0F8EF10F081BABDEF96
:1027700013F05EEC23F0E9EF14F0D7D77252D8A42F
:10278000C4EF13F0040E726E050E725CD8A4CBEF8A
:1027900013F0010E726E010E725CD8A4D8EF13F024
:1027A00000EC14F0656A0BEC14F0656A29EC14F087
:1027B000020E725CD8A4E5EF13F000EC14F0656A29
:1027C00041EC14F0656A60EC14F0030E725CD8A45E
:1027D000F2EF13F000EC14F0656A79EC14F0656A1E
:1027E00098EC14F0040E725CD8A4FFEF13F000EC28
:1027F00014F0656AB1EC14F0656AD0EC14F01200C4
:10280000010E656E0BEC14F041EC14F079EC14F051
:10281000B1EC14F01200436A446A97EC24F0310ED4
:102820004D6E2E0E4E6E560E4F6E2E0E506E720E5A
:10283000516E650E526E660E536E200E546E556EBE
:10284000566E576E586E596E5A6E5B6A61EC24F084
:102850001200320E436E446A97EC24F000EE4DF005
:10286000020E016E1FC123F01EC122F01DC121F016
:102870001CC120F0010E4BEC00F0EF6A61EC24F07B
:102880001200436A010E446E97EC24F0320E4D6E36
:102890002E0E4E6E430E4F6E2E0E506E640E516E07
:1028A000690E526E760E536E200E546E556E566E35
:1028B000576E586E596E5A6E5B6A61EC24F01200C6
:1028C000320E436E010E446E97EC24F000EE4DF094
:1028D000020E016E00C123F0FFC022F0FEC021F005
:1028E000FDC020F0010E4BEC00F0EF6A61EC24F02B
:1028F0001200436A020E446E97EC24F0330E4D6EC4
:102900002E0E4E6E560E4F6E2E0E506E6D0E516E7A
:10291000610E526E780E536E200E546E556E566ECA
:10292000576E586E596E5A6E5B6A61EC24F0120055
:10293000320E436E020E446E97EC24F000EE4DF022
:10294000020E016E17C123F016C122F015C121F04D
:1029500014C120F0010E4BEC00F0EF6A61EC24F0A2
:102960001200436A030E446E97EC24F0340E4D6E51
:102970002E0E4E6E560E4F6E2E0E506E6D0E516E0A
:10298000690E526E6E0E536E200E546E556E566E5C
:10299000576E586E596E5A6E5B6A61EC24F01200E5
:1029A000320E436E030E446E97EC24F000EE4DF0B1
:1029B000020E016E04C123F003C122F002C121F016
:1029C00001C120F0010E4BEC00F0EF6A61EC24F045
:1029D000120092EC2DF03EC015F03D503CEC01F0A1
:1029E000010E725CD8A4FDEF14F01FC11BF11EC1D3
:1029F0001AF11DC119F11CC118F1020E725CD8A4A4
:102A00000AEF15F000C11BF1FFC01AF1FEC019F169
:102A1000FDC018F1030E725CD8A417EF15F017C1B2
:102A20001BF116C11AF115C119F114C118F1040EE8
:102A3000725CD8A424EF15F004C11BF103C11AF194
:102A400002C119F101C118F181BC4AEF15F05EEC29
:102A500023F0CD0E316ECC0E306E4C0E2F6E7B0EF1
:102A60002E6E1BC12DF01AC12CF019C12BF018C10C
:102A70002AF08FEC02F02DC01BF12CC01AF12BC0F4
:102A800019F12AC018F1D9EC15F03EC015F03D50EF
:102A90003CEC01F081B870EF15F05EEC23F0CD0E48
:102AA0002D6ECC0E2C6E4C0E2B6E7B0E2A6E1BC127
:102AB00031F01AC130F019C12FF018C12EF091EC8D
:102AC00002F02DC01BF12CC01AF12BC019F12AC045
:102AD00018F1D9EC15F03EC015F03D503CEC01F07A
:102AE00081BE77EF15F05EEC23F0F8EF10F081BABD
:102AF000BFEF15F05EEC23F0680EA96EFD51E2EC1D
:102B000000F0FE51E2EC00F0FF51E2EC00F00101B8
:102B10000051E2EC00F06C0EA96E0151E2EC00F005
:102B20000251E2EC00F00351E2EC00F00451E2EC5F
:102B300000F0700EA96E1451E2EC00F01551E2ECB9
:102B400000F01651E2EC00F01751E2EC00F0740EC8
:102B5000A96E1C51E2EC00F01D51E2EC00F01E5198
:102B6000E2EC00F01F51E2EC00F0F80EA96E7D0ED1
:102B7000E2EC00F00001B4EC18F08AEF13F0316AD7
:102B8000C00E306E7F0E2F6E880E2E6E1FC12DF080
:102B90001EC12CF01DC12BF01CC12AF023EC03F048
:102BA0002DC06DF02CC06CF02BC06BF02AC06AF009
:102BB0004BD7010E725CD8A4E9EF15F01BC11FF1D1
:102BC0001AC11EF119C11DF118C11CF1BEEC13F0A0
:102BD0001200020E725CD8A4F9EF15F01BC100F1CF
:102BE0001AC1FFF019C1FEF018C1FDF0BEEC13F0E0
:102BF0001200030E725CD8A409EF16F01BC117F186
:102C00001AC116F119C115F118C114F1BEEC13F077
:102C10001200040E725CD8A419EF16F01BC104F167
:102C20001AC103F119C102F118C101F1BEEC13F090
:102C30001200E90EC26EC16A0A0EEFEC00F020C06D
:102C40002AF021C02BF0DBEC03F02DC069F02CC082
:102C500068F02BC067F02AC066F0E80EC26EFC0E6A
:102C6000C16E640E48EC01F069C031F068C030F00C
:102C700067C02FF066C02EF06DC02DF06CC02CF038
:102C80006BC02BF06AC02AF08BEC03F02DC023F050
:102C90002CC022F02BC021F02AC020F023C031F03C
:102CA00022C030F021C02FF020C02EF000C12DF046
:102CB000FFC02CF0FEC02BF0FDC02AF08BEC03F01F
:102CC0002DC071F02CC070F02BC06FF02AC06EF0D8
:102CD000020E436E446A97EC24F094988288456A09
:102CE000466A4652D8A489EF17F0100E455CD8B05A
:102CF00089EF17F071C02DF070C02CF06FC02BF071
:102D00006EC02AF004C131F003C130F002C12FF0CF
:102D100001C12EF017EC02F00108D8B4A1EF16F0B3
:102D20002F0E0F6E440E0E6E45500E24F66E46505A
:102D30000F20F76EA66AA68E0800F5CF0CF00CC027
:102D40004DF071C02DF070C02CF06FC02BF06EC034
:102D50002AF004C131F003C130F002C12FF001C1EB
:102D60002EF017EC02F0326E71C02DF070C02CF016
:102D70006FC02BF06EC02AF00FC131F00EC130F0E1
:102D80000DC12FF00CC12EF053EC02F03216D8B466
:102D9000DBEF16F02F0E0F6E560E0E6E45500E2402
:102DA000F66E46500F20F76EA66AA68E0800F5CF85
:102DB0000CF00CC04DF071C02DF070C02CF06FC045
:102DC0002BF06EC02AF00FC131F00EC130F00DC1F2
:102DD0002FF00CC12EF0DFEC01F0326E71C02DF03F
:102DE00070C02CF06FC02BF06EC02AF013C131F010
:102DF00012C130F011C12FF010C12EF053EC02F0CF
:102E00003216D8B415EF17F02F0E0F6E680E0E6E37
:102E100045500E24F66E46500F20F76EA66AA68E19
:102E20000800F5CF0CF00CC04DF071C02DF070C053
:102E30002CF06FC02BF06EC02AF013C131F012C11C
:102E400030F011C12FF010C12EF0DFEC01F0326E26
:102E500071C02DF070C02CF06FC02BF06EC02AF046
:102E600017C131F016C130F015C12FF014C12EF08A
:102E700053EC02F03216D8B44FEF17F02F0E0F6E4E
:102E80007A0E0E6E45500E24F66E46500F20F76EE9
:102E9000A66AA68E0800F5CF0CF00CC04DF017C145
:102EA0002DF016C12CF015C12BF014C12AF071C001
:102EB00031F070C030F06FC02FF06EC02EF017EC04
:102EC00002F00108D8B476EF17F02F0E0F6E8C0EBB
:102ED0000E6E45500E24F66E46500F20F76EA66A11
:102EE000A68E0800F5CF0CF00CC04DF0820E056EDA
:102EF000080E0A6E820E066E040E076E010E0B6E31
:102F00004D50106E05EC01F0452AD8B4462AD8A4DD
:102F1000E8D671C02DF070C02CF06FC02BF06EC0E1
:102F20002AF004C131F003C130F002C12FF001C119
:102F30002EF017EC02F00108D8B4A1EF17F0D0EC96
:102F400017F012007E424242424242424242424214
:102F5000427E243C12007E7A7262424242424242E7
:102F60004242427E243C12007E7A766E5E7A726223
:102F700042424242427E243C12007E7A766E5E7A63
:102F8000766E5E7A7262427E243C12007E7A766EA3
:102F90005E7A766E5E7A766E5E7E243C1200120059
:102FA0000101072B000E082309230A230ABF14D0AE
:102FB0000A530001D8A4EDEF17F0010109510001F7
:102FC000D8A4EDEF17F0F40E0101075D010E0859CA
:102FD0000001D8B0EDEF17F0120001010A6B096B88
:102FE000086B076B00010EEC18F0DEEC22F0320EDD
:102FF0003BEC01F0DEEC22F0320E3BEC01F0DEECBB
:1030000022F0320E3BEC01F0C831D8B00DEF18F0D1
:10301000030E156EE80E3CEC01F01200020E436E3A
:10302000446A97EC24F094988288456A466A46522E
:10303000D8A444EF18F0130E455CD8B044EF18F054
:10304000300E0F6E8A0E0E6E45500E24F66E4650F0
:103050000F20F76EA66AA68E0800F5CF0CF00CC004
:103060004DF0820E056E080E0A6E820E066E040E7C
:10307000076E010E0B6E4D50106E05EC01F0452AE7
:10308000D8B4462AD8A4D3D71200007E4040003CD2
:1030900042423C003E403E403E0000000000120024
:1030A000680EDCEC00F0FD6FDDEC00F0FE6FDDEC97
:1030B00000F0FF6FDDEC00F00101006F6C0EDCEC46
:1030C00000F0016FDDEC00F0026FDDEC00F0036F4B
:1030D000DDEC00F0046F700EDCEC00F0146FDDEC42
:1030E00000F0156FDDEC00F0166FDDEC00F0176FEF
:1030F000740EDCEC00F01C6FDDEC00F01D6FDDECFD
:1031000000F01E6FDDEC00F01F6FF80EDCEC00F03D
:10311000246F00017D0E0101245D0001D8B4B3EFDE
:1031200018F00101006B0001FF6BFE6B800EFD6F5C
:103130000101046B036B600E026F810E016F176B50
:10314000166B100E156F820E146F140E6D6E280E16
:103150006C6E200E6B6E770E6A6E1F6B1E6B200EF0
:103160001D6F810E1C6F0001140E6D6E280E6C6EAB
:10317000200E6B6E770E6A6E17C12DF016C12CF003
:1031800015C12BF014C12AF004C131F003C130F095
:1031900002C12FF001C12EF08FEC02F02DC023F000
:1031A0002CC022F02BC021F02AC020F0316A306AF6
:1031B000400E2F6E800E2E6E23C02DF022C02CF0FC
:1031C00021C02BF020C02AF023EC03F02DC00FF11A
:1031D0002CC00EF12BC00DF12AC00CF10FC131F043
:1031E0000EC130F00DC12FF00CC12EF004C12DF036
:1031F00003C12CF002C12BF001C12AF091EC02F0C6
:103200002DC00FF12CC00EF12BC00DF12AC00CF116
:1032100017C12DF016C12CF015C12BF014C12AF0E6
:1032200004C131F003C130F002C12FF001C12EF012
:103230008FEC02F02DC023F02CC022F02BC021F027
:103240002AC020F0316A306A400E2F6E800E2E6E3A
:1032500023C02DF022C02CF021C02BF020C02AF07A
:1032600023EC03F02DC013F12CC012F12BC011F18F
:103270002AC010F113C123F012C122F011C121F0B4
:103280000101103D02D037821051206E23C031F071
:1032900022C030F021C02FF020C02EF004C12DF04C
:1032A00003C12CF002C12BF001C12AF091EC02F015
:1032B0002DC013F12CC012F12BC011F12AC010F156
:1032C000000112007FEC24F0436A446A97EC24F07A
:1032D000200E4D6E4E6E4F6E430E506E6F0E516E41
:1032E0006E0E526E740E536E720E546E610E556EEB
:1032F000730E566E740E576E200E586E596E5A6EBF
:103300005B6A61EC24F0F8EC19F092EC2DF0BEEC65
:1033100019F03EC015F03D503CEC01F081B89BEF38
:1033200019F05EEC23F001010B2B0001BEEC19F04B
:10333000B7EC23F0C7D781BCA8EF19F05EEC23F0FF
:1033400001010B070001BEEC19F0B7EC23F0BAD76E
:1033500081BEAFEF19F05EEC23F0F8EF10F081BA08
:10336000BDEF19F05EEC23F0640EA96E01010B5164
:10337000E2EC00F00001F8EF10F0D0D7640E01018C
:103380000B5D0001D8B0C8EF19F0640E01010B6F9E
:103390000001FB0E01010B5D0001D8A0D3EF19F075
:1033A000FA0E01010B6F0001D7EC19F01200436A0D
:1033B000020E446E97EC24F0200E4D6E4E6E4F6E52
:1033C000506E516E526A61EC24F00A0E436E020E8A
:1033D000446E97EC24F000EE4DF0020E016E0101F8
:1033E0000B5119EC00F0EF6A000161EC24F01200BF
:1033F000436A010E446E97EC24F094988288456AE3
:10340000466A4652D8A42EEF1AF0FD0E455CD8B09D
:103410002EEF1AF0340E0F6E640E0E6E45500E2411
:10342000F66E46500F20F76EA66AA68E0800F5CFFE
:103430000CF00CC04DF0820E056E080E0A6E820E66
:10344000066E040E076E010E0B6E4D50106E05ECED
:1034500001F0452AD8B4462AD8A4D3D7960E3BEC1F
:1034600001F0120000000000000000000000000059
:10347000000000000000000000000000000000004C
:10348000000000000000000000000000000000003C
:10349000408000008080C0C0F0C0C08080008040BC
:1034A000000000000000000000000000000000001C
:1034B000000000000000000000000000000000000C
:1034C00000000000000000000000000000000000FC
:1034D00000000000000000000000000000000000EC
:1034E0000000002020F8FFFFFFFFFFFFFF000001AA
:1034F0000107FEF82020000000000000000000008E
:1035000000000000000000000000000000000000BB
:1035100000000000000000000000000000000000AB
:10352000000000000000000000000000000000009B
:10353000000000000000000000100B070F0F1F1F0D
:103540007F18180C0C070B10000000000000000092
:10355000000000000000000000000000000000006B
:1035600012007FEC24F0436A446A97EC24F0430E87
:103570004D6E610E4E6E6C0E4F6E2E0E506E200E06
:10358000516E630E526E610E536E700E546E610E6C
:10359000556E630E566E690E576E740E586E6F0E32
:1035A000596E720E5A6E5B6A61EC24F092EC2DF04B
:1035B00042EC1BF03EC015F03D503CEC01F081B8F0
:1035C00002EF1BF05EEC23F02D6A2C6A2B6A7F0E53
:1035D0002A6E9EC031F09DC030F09CC02FF09BC081
:1035E0002EF091EC02F02DC09EF02CC09DF02BC06F
:1035F0009CF02AC09BF042EC1BF03EC015F03D5001
:103600003CEC01F081BC25EF1BF05EEC23F0316A4D
:10361000306A2F6A7F0E2E6E9EC02DF09DC02CF05A
:103620009CC02BF09BC02AF08FEC02F02DC09EF0C6
:103630002CC09DF02BC09CF02AC09BF042EC1BF0EC
:103640003EC015F03D503CEC01F081BE2CEF1BF06C
:103650005EEC23F0F8EF10F081BA41EF1BF05EEC66
:1036600023F0010EA96E9B51E2EC00F09C51E2ECBC
:1036700000F09D51E2EC00F09E51E2EC00F0F8EF1A
:1036800010F09DD79CBF0BD0000E9E5D000E9D5983
:103690007A0E9C59870E9B59D8B055EF1BF09E6B44
:1036A0009D6B7A0E9C6F870E9B6FD8969CBFD886B9
:1036B000D8B66DEF1BF0010E9E5D800E9D593B0E3E
:1036C0009C59890E9B59D8A06DEF1BF09E6B800E04
:1036D0009D6F3B0E9C6F890E9B6F70EC1BF0120070
:1036E000436A020E446E97EC24F0200E4D6E4E6E2F
:1036F0004F6E506E516E526E536E546E556E700E0C
:10370000566E460E576E200E586E596E5A6E5B6A94
:1037100061EC24F00F0E436E020E446E97EC24F021
:1037200000EE4DF0020E016E9EC023F09DC022F00F
:103730009CC021F09BC020F0010E4BEC00F0EF6A22
:1037400061EC24F01200C831D8A0B4EF1BF0D89679
:10375000C8A1D886D8B6B4EF1BF0A6EC27F03EC0BF
:1037600015F03D503CEC01F0C831D8B0BFEF1BF074
:10377000DBEC28F03EC015F03D503CEC01F081B888
:10378000D5EF1BF05EEC23F0C881A6EC27F0030E0A
:10379000156EE80E3CEC01F00A0EA96EE86AC8B19D
:1037A000010EE2EC00F0F8EF10F081BAEBEF1BF045
:1037B0005EEC23F0C891DBEC28F0030E156EE80EEA
:1037C0003CEC01F00A0EA96EE86AC8B1010EE2EC09
:1037D00000F0F8EF10F0D3D7C831E832D8A0F8EFF6
:1037E0001BF010EC2AF03EC015F03D503CEC01F00F
:1037F000C831E832D8B004EF1CF045EC2BF03EC0E5
:1038000015F03D503CEC01F081B81BEF1CF05EEC74
:1038100023F0C88310EC2AF08180030E156EE80EA9
:103820003CEC01F00B0EA96EE86AC8B3010EE2ECA5
:1038300000F0F8EF10F081BA32EF1CF05EEC23F0EC
:10384000C89345EC2BF08190030E156EE80E3CEC0E
:1038500001F00B0EA96EE86AC8B3010EE2EC00F0AD
:10386000F8EF10F0D1D7C831E832D8A049EF1CF0FA
:10387000C89345EC2BF08190030E156EE80E3CECDE
:1038800001F00B0EA96EE86AC8B3010EE2EC00F07D
:103890001200C831E832D8B05FEF1CF0C88310ECDA
:1038A0002AF08180030E156EE80E3CEC01F00B0E41
:1038B000A96EE86AC8B3010EE2EC00F012007FECDA
:1038C00024F0436A446A97EC24F0200E4D6E4E6E4D
:1038D0004F0E4F6E730E506E630E516E690E526E28
:1038E0006C0E536E546E610E556E740E566E6F0EE6
:1038F000576E720E586E200E596E5A6E5B6A61ECEE
:1039000024F092EC2DF03EC015F03D503CEC01F05F
:1039100081B899EF1CF05EEC23F0C42B000EC52398
:10392000C623C7232FEC1DF03EC015F03D503CECE4
:1039300001F081BCAAEF1CF05EEC23F0C407000E7E
:10394000C55BC65BC75B2FEC1DF03EC015F03D505C
:103950003CEC01F081BEB1EF1CF05EEC23F0F8EF1F
:1039600010F081BAC6EF1CF05EEC23F00C0EA96ECD
:10397000C451E2EC00F0C551E2EC00F0C651E2ECBB
:1039800000F0C751E2EC00F0F8EF10F0656A436A0E
:10399000030E446E97EC24F0200E4D6E4E6E4F6E6B
:1039A000506E516E526E536E546E556E566E4B0E77
:1039B000576E200E586E596E5A6E5B6A61EC24F099
:1039C000656A190E436E030E446E97EC24F000EE08
:1039D0004DF0020E016E096AC7C023F0C6C022F086
:1039E000C5C021F0C4C020F0ACEC00F0EF6A61EC7F
:1039F00024F03EEC10F0436A010E446E97EC24F084
:103A0000200E4D6E4E6E4F6E506E516E526E536E56
:103A1000546E556E566E480E576E7A0E586E200EC6
:103A2000596E5A6E5B6E5C6A61EC24F00F0E436E49
:103A3000010E446E97EC24F000EE4DF0020E016E84
:103A4000096A7AC023F079C022F078C021F077C0EB
:103A500020F0ACEC00F0EF6A61EC24F059D7C7BF5E
:103A60000FD0C753D8A446EF1DF0C651D8A446EFD7
:103A70001DF0840EC45D030EC559D8B046EF1DF08D
:103A8000C76BC66B030EC56F840EC46FD896C7BFD5
:103A9000D886D8B65DEF1DF0C75309E1C65107E1DE
:103AA0004D0EC45D040EC559D8A05DEF1DF0C76B67
:103AB000C66B040EC56F4C0EC46F120043EC38F099
:103AC000030E156EE80E3CEC01F0A8EC1DF078EC4E
:103AD00039F0030E156EE80E3CEC01F0A8EC1DF079
:103AE000ADEC3AF0030E156EE80E3CEC01F0A8ECDC
:103AF0001DF0E2EC3BF0030E156EE80E3CEC01F01D
:103B0000A8EC1DF017EC3DF0030E156EE80E3CEC32
:103B100001F0A8EC1DF078EC39F0030E156EE80EFC
:103B20003CEC01F0A8EC1DF04CEC3EF0030E156EE1
:103B3000E80E3CEC01F0A8EC1DF0E2EC3BF0030ECB
:103B4000156EE80E3CEC01F0A8EC1DF0F8EF10F05B
:103B500081BEACEF1DF0120081BCB0EF1DF0120071
:103B600081BAB4EF1DF0120081B8B8EF1DF0120059
:103B7000EFD74B0E436E446A97EC24F0520E4D6E15
:103B8000200E4E6E4F6E506A61EC24F0436A020EB6
:103B9000446E97EC24F0200E4D6E4E6E4F6E506EBC
:103BA000516E570E526E720E536E690E546E740E35
:103BB000556E650E566E200E576E586E596E5A6EC3
:103BC0005B6E5C6A61EC24F082AEE8EF1DF0F58973
:103BD00082BEECEF1DF0F599F0C0F4F0EFC0F3F009
:103BE000EEC0F2F0EDC0F1F0ECC0F0F0EBC0EFF0A1
:103BF000EAC0EEF0E9C0EDF0E8C0ECF0E7C0EBF0B1
:103C0000E6C0EAF0E5C0E9F0E4C0E8F0E3C0E7F0C0
:103C1000E2C0E6F0E1C0E5F0E0C0E4F0DFC0E3F0D0
:103C2000DEC0E2F0DDC0E1F0DCC0E0F0DBC0DFF0E0
:103C3000DAC0DEF0D9C0DDF0D8C0DCF0D7C0DBF0F0
:103C4000D6C0DAF0D5C0D9F0D4C0D8F0D3C0D7F000
:103C5000D2C0D6F0D1C0D5F0D0C0D4F0CFC0D3F010
:103C6000CEC0D2F0CDC0D1F0F9C0D0F0F8C0CFF0C6
:103C7000F7C0CEF0F6C0CDF0F587F5A5F597F58540
:103C8000F5A3F595F583F5A1F593F581C8AFF59109
:103C9000C88FC8ADC89FC88DC8ABC89DC88BC8A900
:103CA000C89BC889C8A7C899C887C8A5C897C88528
:103CB000F5A9C89522EC1FF03EC015F03D503CEC34
:103CC00001F04EEF05F0140EDCEC00F0CD6FDDECF2
:103CD00000F0CE6FDDEC00F0CF6FDDEC00F0D06FC8
:103CE000180EDCEC00F0D16FDDEC00F0D26FDDECF3
:103CF00000F0D36FDDEC00F0D46F1C0EDCEC00F0B4
:103D0000D56FDDEC00F0D66FDDEC00F0D76FDDECA9
:103D100000F0D86F200EDCEC00F0D96FDDEC00F085
:103D2000DA6FDDEC00F0DB6FDDEC00F0DC6F240E11
:103D3000DCEC00F0DD6FDDEC00F0DE6FDDEC00F0C0
:103D4000DF6FDDEC00F0E06F280EDCEC00F0E16FDF
:103D5000DDEC00F0E26FDDEC00F0E36FDDEC00F095
:103D6000E46F2C0EDCEC00F0E56FDDEC00F0E66FAC
:103D7000DDEC00F0E76FDDEC00F0E86F300EDCEC1E
:103D800000F0E96FDDEC00F0EA6FDDEC00F0EB6FC6
:103D9000DDEC00F0EC6F340EDCEC00F0ED6FDDECF0
:103DA00000F0EE6FDDEC00F0EF6FDDEC00F0F06F97
:103DB000380EDCEC00F0F16FDDEC00F0F26FDDECC2
:103DC00000F0F36FDDEC00F0F46F3C0EDCEC00F083
:103DD000C885E8A0C895400EDCEC00F0C887E8A0D4
:103DE000C897440EDCEC00F0C889E8A0C899480EDA
:103DF000DCEC00F0C88BE8A0C89B4C0EDCEC00F0BB
:103E0000C88DE8A0C89D500EDCEC00F0C88FE8A07B
:103E1000C89F540EDCEC00F0F581E8A0F591580E37
:103E2000DCEC00F0F583E8A0F5935C0EDCEC00F030
:103E3000F585E8A0F595600EDCEC00F0F587E8A0CC
:103E4000F5971200140EA96ECD51E2EC00F0CE51A0
:103E5000E2EC00F0CF51E2EC00F0D051E2EC00F0E7
:103E6000180EA96ED151E2EC00F0D251E2EC00F054
:103E7000D351E2EC00F0D451E2EC00F01C0EA96E3C
:103E8000D551E2EC00F0D651E2EC00F0D751E2EC73
:103E900000F0D851E2EC00F0200EA96ED951E2EC0E
:103EA00000F0DA51E2EC00F0DB51E2EC00F0DC5122
:103EB000E2EC00F0240EA96EDD51E2EC00F0DE51E0
:103EC000E2EC00F0DF51E2EC00F0E051E2EC00F057
:103ED000280EA96EE151E2EC00F0E251E2EC00F0B4
:103EE000E351E2EC00F0E451E2EC00F02C0EA96E9C
:103EF000E551E2EC00F0E651E2EC00F0E751E2ECD3
:103F000000F0E851E2EC00F0300EA96EE951E2EC6D
:103F100000F0EA51E2EC00F0EB51E2EC00F0EC5181
:103F2000E2EC00F0340EA96EED51E2EC00F0EE513F
:103F3000E2EC00F0EF51E2EC00F0F051E2EC00F0C6
:103F4000380EA96EF151E2EC00F0F251E2EC00F013
:103F5000F351E2EC00F0F451E2EC00F03C0EA96EFB
:103F6000E86AC8B5010EE2EC00F0400EA96EE86AFE
:103F7000C8B7010EE2EC00F0440EA96EE86AC8B9B9
:103F8000010EE2EC00F0480EA96EE86AC8BB010E13
:103F9000E2EC00F04C0EA96EE86AC8BD010EE2EC3E
:103FA00000F0500EA96EE86AC8BF010EE2EC00F006
:103FB000540EA96EE86AF5B1010EE2EC00F0580E5D
:103FC000A96EE86AF5B3010EE2EC00F05C0EA96E92
:103FD000E86AF5B5010EE2EC00F0600EA96EE86A41
:103FE000F5B7010EE2EC00F012007FEC24F006ECD5
:103FF0002DF0436A446A97EC24F04D0E4D6E650E29
:104000004E6E6D0E4F6E6F0E506E720E516E790EBB
:10401000526E200E536E546E556E566E576E586E1D
:10402000596E5A6E5B6A61EC24F0010E726E140ECA
:10403000FA6F3C0EFB6F50EC20F084EC20F03EC099
:1040400015F03D503CEC01F081BC36EF20F05EEC09
:1040500023F0722A040EFA27FB2750EC20F084ECA0
:1040600020F03EC015F03D503CEC01F081B848EF27
:1040700020F05EEC23F07206040EFA5FFB5F50EC5A
:1040800020F084EC20F03EC015F03D503CEC01F0F7
:1040900081BE4FEF20F05EEC23F0F8EF10F0D4D7A4
:1040A0007252D8A45AEF20F0010E726E140EFA6FFD
:1040B0003C0EFB6F0B0E725CD8A465EF20F00A0E6D
:1040C000726E380EFA6F600EFB6F3C0E436E446AE0
:1040D00097EC24F0230E4D6E200E4E6E4F6E506EF8
:1040E000516E526A61EC24F0440E436E446A97ECC0
:1040F00024F000EE4DF0020E016E725019EC00F04B
:10410000EF6A61EC24F01200FA51DCEC00F0F66F7B
:10411000DDEC00F0F76FDDEC00F0F86FDDEC00F0A7
:10412000F96FFB51DCEC00F0F589E8A0F599D89621
:10413000F5A9D886D8B69FEF20F0A7EF20F0D89643
:10414000F5B9D886D8B6A7EF20F059EF21F0436A29
:10415000010E446E97EC24F0200E4D6E4E6E4F6EA5
:10416000506E516E526E536E546E556E566E576E43
:10417000586E700E596E460E5A6E5B6A61EC24F0F2
:10418000436A010E446E97EC24F000EE4DF0020EEF
:10419000016EF9C023F0F8C022F0F7C021F0F6C09C
:1041A00020F0010E4BEC00F0EF6A61EC24F0436A62
:1041B000020E446E97EC24F0200E4D6E4E6E4F6E44
:1041C000506E516E526E536E546E556E566E576EE3
:1041D000586E6E0E596E460E5A6E5B6A61EC24F094
:1041E000436A020E446E97EC24F000EE4DF0020E8E
:1041F000016E316A306A7A0E2F6E880E2E6EF9C00B
:104200002DF0F8C02CF0F7C02BF0F6C02AF023EC0C
:1042100003F02DC023F02CC022F02BC021F02AC0C7
:1042200020F0060E4BEC00F0EF6A61EC24F0436ADC
:10423000030E446E97EC24F0200E4D6E4E6E4F6EC2
:10424000506E516E526E536E546E556E566E576E62
:10425000586E750E596E460E5A6E5B6A61EC24F00C
:10426000436A030E446E97EC24F000EE4DF0020E0C
:10427000016E316A240E306E740E2F6E920E2E6E09
:10428000F9C02DF0F8C02CF0F7C02BF0F6C02AF0E2
:1042900023EC03F02DC023F02CC022F02BC021F022
:1042A0002AC020F0060E4BEC00F0EF6A61EC24F01F
:1042B0001200436A010E446E97EC24F0200E4D6EFE
:1042C0004E6E4F6E506E516E526E536E546E556EF2
:1042D000566E576E586E596E5A6E5B6A61EC24F0DA
:1042E000436A020E446E97EC24F0200E4D6E4E6E23
:1042F0004F6E506E516E526E536E546E556E566EBA
:10430000576E586E6E0E596E480E5A6E5B6A61ECAF
:1043100024F0436A020E446E97EC24F000EE4DF058
:10432000020E016E2D6A2C6A7A0E2B6E880E2A6E92
:10433000F9C031F0F8C030F0F7C02FF0F6C02EF021
:104340008BEC03F02DC023F02CC022F02BC021F009
:104350002AC020F0010E4BEC00F0EF6A61EC24F073
:10436000436A030E446E97EC24F0200E4D6E4E6EA1
:104370004F6E506E516E526E536E546E556E566E39
:10438000576E586E750E596E480E5A6E5B6A61EC28
:1043900024F0436A030E446E97EC24F000EE4DF0D7
:1043A000020E016EF9C023F0F8C022F0F7C021F030
:1043B000F6C020F0030E4BEC00F0EF6A61EC24F045
:1043C0001200436A446A97EC24F094988288456A04
:1043D000466A4652D8A416EF22F0300E455CD8B09B
:1043E00016EF22F0440E0F6E2E0E0E6E45500E2468
:1043F000F66E46500F20F76EA66AA68E0800F5CF1F
:104400000CF00CC04DF0820E056E080E0A6E820E86
:10441000066E040E076E010E0B6E4D50106E05EC0D
:1044200001F0452AD8B4462AD8A4D3D712007F0178
:1044300001017F7901017F007C74545C007C0404DD
:104440007C74047C007C74447C007C7404001C70CC
:10445000701C0000000000000000000000001200BE
:10446000130E436E446A97EC24F094988288456A50
:10447000466A4652D8A466EF22F0380E455CD8B0A2
:1044800066EF22F0440E0F6ECE0E0E6E45500E24D7
:10449000F66E46500F20F76EA66AA68E0800F5CF7E
:1044A0000CF00CC04DF0820E056E080E0A6E820EE6
:1044B000066E040E076E010E0B6E4D50106E05EC6D
:1044C00001F0452AD8B4462AD8A4D3D71200000058
:1044D00000000000000000000000000000080808C4
:1044E000080808087F7F007F7F0808080808080878
:1044F00000000000000000000000000000000000BC
:104500000000000000001200130E436E446A97EC96
:1045100024F094988288456A466A4652D8A4BAEF35
:1045200022F0380E455CD8B0BAEF22F0450E0F6E7F
:10453000760E0E6E45500E24F66E46500F20F76E26
:10454000A66AA68E0800F5CF0CF00CC04DF0820EC6
:10455000056E080E0A6E820E066E040E076E010EC0
:104560000B6E4D50106E05EC01F0452AD8B4462A6A
:10457000D8A4D3D712000000000040404040700C87
:1045800002020101010102020C700C020201010190
:104590000102020C700C02020101010102020C7006
:1045A000404040400000000000000000000000000B
:1045B000000000000000000000001200C831D8A078
:1045C000EAEF22F0D896C8A1D886D8B6EAEF22F052
:1045D000EBEF22F01200C36BC26BC16BC06BC3BFA9
:1045E0000BD0C151C211C311D8A40FEF23F0150E87
:1045F000C05DD8B00FEF23F08186050E116EDC0E82
:1046000049EC01F08196050E116EDC0E49EC01F0CB
:10461000C02B000EC123C223C323D8A0E0D71E0E97
:104620003BEC01F0C36BC26BC16BC06BC3BF0BD063
:10463000C151C211C311D8A436EF23F0150EC05DCD
:10464000D8B036EF23F08186050E116EDC0E49ECF2
:1046500001F08196050E116EDC0E49EC01F0C02BC5
:10466000000EC123C223C323D8A0E0D71E0E3BEC0B
:1046700001F0C36BC26BC16BC06BC3BF0BD0C15128
:10468000C211C311D8A45DEF23F0150EC05DD8B0E0
:104690005DEF23F08186050E116EDC0E49EC01F012
:1046A0008196050E116EDC0E49EC01F0C02B000E58
:1046B000C123C223C323D8A0E0D71200C831D8A099
:1046C0006AEF23F0D896C8A1D886D8B66AEF23F04F
:1046D0006BEF23F01200C36BC26BC16BC06BC3BF27
:1046E0000BD0C151C211C311D8A48FEF23F0150E06
:1046F000C05DD8B08FEF23F08186050E116EDC0E01
:1047000049EC01F08196050E116EDC0E49EC01F0CA
:10471000C02B000EC123C223C323D8A0E0D7140EA0
:104720003BEC01F0C36BC26BC16BC06BC3BF0BD062
:10473000C151C211C311D8A4B6EF23F0150EC05D4C
:10474000D8B0B6EF23F08186030E116EE80E49EC67
:1047500001F08196030E116EE80E49EC01F0C02BBA
:10476000000EC123C223C323D8A0E0D71200010E3C
:10477000656E949A829ADBEC23F07FEC24F0140EA1
:104780003BEC01F094988298820E056E080E0A6E3A
:10479000820E066E040E076E010E0B6E210E106E59
:1047A00005EC01F00BC110F005EC01F0200E106ECD
:1047B00005EC01F01200949C829C140E3BEC01F07D
:1047C000949C828C949A829A94988298210E626E1C
:1047D000FFEC23F0C80E626EFFEC23F0080E626E51
:1047E000FFEC23F0130E626EFFEC23F0200E626EDE
:1047F000FFEC23F00C0E626EFFEC23F01200820E31
:10480000056E080E0A6E820E066E040E076E010E0D
:104810000B6E62C010F005EC01F012006250060D44
:10482000F3CF40F0F4CF41F03F6A060E3F5CD8B0C2
:104830003CEF24F0490E0D6EEA0E0C6E40500C2435
:10484000206E41500D20216E3F502024F66E000E48
:104850002120F76EA66AA68E0800F5CF62F0655299
:10486000D8A434EF24F0621E00EE47F03F5062C03F
:10487000EBFF3F2AD8A4D9D794988288820E056E80
:10488000080E0A6E820E066E040E076E010E0B6E87
:104890004750106E05EC01F04850106E05EC01F029
:1048A0004950106E05EC01F04A50106E05EC01F015
:1048B0004B50106E05EC01F04C50106E05EC01F001
:1048C0001200426A150E425CD8B076EF24F000EE7A
:1048D0004DF04250EB50626E6252D8A472EF24F059
:1048E00076EF24F09BDF422AD8A4ECD7010E656E48
:1048F000120094988298C80E626E81DF120092ECCA
:1049000024F094988288010E3F6EFD0E3F5CD8B073
:1049100091EF24F0626A73DF626A71DF3F2AD8A4E4
:10492000F4D71200436A446A97EC24F0120094987A
:104930008298400E4410626E62DF800E4310626EF9
:104940005EDF12009498829844C020F0216A44C02F
:1049500024F0256A253224322532243225322432AD
:104960001F0E2516243625362436253624362536C0
:10497000F80E24162450205E2550215A2004636E20
:10498000400E206E216A44C024F0256A2406000EE1
:10499000255A2532243225322432253224321F0E64
:1049A000251620502410626E2ADFFF0E4324206E4D
:1049B000216AFF0E2122800E2010626E20DF949863
:1049C0008288820E056E080E0A6E820E066E040E36
:1049D000076E010E0B6E106E635004E0D890103617
:1049E000E82EFCD705EC01F01200000000000000EA
:1049F000FFFFFFFFFFFF07070700000000000007A1
:104A00000707E0E0E0000000000000E0E0E0FFFF5A
:104A1000FF000000000000FFFFFF07070707070770
:104A2000E0E0E0E0E0E0E0E0E0070707070707E09C
:104A3000E0E0FFFFFFE0E0E0E0E0E0FFFFFF07076E
:104A400007FFFFFFFFFFFF07070755AA55AA55AA53
:104A5000AA55AA55AA550101010101018080808053
:104A60008080FF00000000000000000000FFFF0148
:104A7000010101010101010101FFFF8080808080AF
:104A80008080808080FF00000000F0F000000000C7
:104A90000F0F0000000000000000000000000000F8
:104AA0000000000000000000000000000000000006
:104AB00000004F000000000700070000147F147F73
:104AC0001400242A7F2A1200231308646200364946
:104AD000552250000005030000001C224100000088
:104AE000000041221C0014083E08140008083E087B
:104AF00008000050300000000808080808000060A6
:104B0000600000002010080402003E5149453E00AC
:104B100000427F4000004261514946002141454B1F
:104B200031001814127F10002745454539003C4AD2
:104B300049493000017109050300364949493600E9
:104B4000064949493E00003636000000005636004E
:104B50000000081422410000141414141400004131
:104B600022140800020151090600324979413E0031
:104B70007E1111117E007F49494936003E41414175
:104B800022007F4141221C007F49494941007F09A1
:104B9000090901003E4149497A007F0808087F0061
:104BA00000417F4100002040413F01007F08142266
:104BB00041007F40404040007F020C027F007F04A4
:104BC00008107F003E4141413E007F09090906006F
:104BD0003E4151215E007F09192946004649494955
:104BE000310001017F0101003F4040403F001F2094
:104BF00040201F003F4038403F006314081463000A
:104C00000708700807006151494543007F41410092
:104C10000000020408102000000041417F0004024F
:104C20000102040040404040400000010204000036
:104C30002054545478007F48444438003844444455
:104C40002000384444487F00385454541800087EEB
:104C5000090102000C5252523E007F080404780001
:104C600000447D400000002040443D007F10284467
:104C7000000000417F4000007C04180478007C089C
:104C8000040478003844444438007C1414140800A8
:104C9000081414187C007C08040408004854545478
:104CA0002000043F444020003C4040207C001C2069
:104CB00040201C003C4030403C0044281028440068
:104CC0000C5050503C004464544C440008364100A1
:104CD000000000007F0000000000413608000008CE
:104CE000040804001FDE94988288456A466A010E13
:104CF000465CD8A084EF26F0D8A4A8EF26F0F80EE2
:104D0000455CD8B0A8EF26F04D0E0F6E520E0E6E19
:104D100045500E24F66E46500F20F76EA66AA68EFA
:104D20000800F5CF0CF00CC04DF0820E056E080E99
:104D30000A6E820E066E040E076E010E0B6E4D504B
:104D4000106E05EC01F0452AD8B4462AD8A4CFD776
:104D50001200000000003058C8A8B870F0F0D0E091
:104D6000C000000000000000000000000000000083
:104D7000000000000080E0F0F8FCFE7FBFFFFFFFB6
:104D8000FEFC7800FEFEFEFEFEFE000000000000BD
:104D9000000000E0F0F8FCFEFE1E1E1E1EFEFEFCE3
:104DA000F8F080000000001E66DE3CF8F0F0F9FF2D
:104DB000FEFF7FDFF7FFE0C0800000000000000082
:104DC000000080E0F0F8FC7EBFDFEF77BBDD7E3FC8
:104DD0001F1F0F0703818080BFBFBFBFBFBF000081
:104DE000808080808080003FBF8FEF8F3F808080F9
:104DF000808F8F0F0F8F8F80808000000000010355
:104E00000206060606040D1B37679F3F7FFFFEFC68
:104E1000F8F0ECFEF6EADFFFFBF5EE1F1B0D0603D4
:104E20000100000000000000003F3C0080BFBC808B
:104E300080BF00003F3E2222223B00808080BFBC1A
:104E4000803F3E2222223B00003F3C000000000049
:104E5000000000000000000000000000000080C111
:104E6000E2F4F973274F9F3F7F7F7E7D79F1E0C0A9
:104E700080000000000000000000000000000000B2
:104E8000FFFFFFFFFFFF8080808080808080007FA9
:104E9000FFFFFFFFFF80808080FEFEFEFEFE7E00A3
:104EA0000000000000000000000080C0E0F0F87C7E
:104EB0003E1F0F070301000000000001020408105C
:104EC00030D83DCFF7FBFDBFFF7F5FBEBC68D0E0B1
:104ED000800000000F0F0F0F0F0F0F0F0F0F0FCFDE
:104EE0000F0F00000103070F0F0F0F0F0F0F0F071A
:104EF0000301000000000000E0F8FC5C6E371F07B3
:104F0000030100000000000000000000000000009D
:104F100000000000003F605FFF9F9E9FB8B0F0E080
:104F2000E101030301000000030C300C03003F0209
:104F30000100013F2100FF1221211E0020003F023D
:104F400001001F2020103F000000120092EC24F00E
:104F500094988288456A466A010E465CD8A0B9EFEB
:104F600027F0D8A4DDEF27F0F80E455CD8B0DDEFD0
:104F700027F04F0E0F6EBC0E0E6E45500E24F66ECF
:104F800046500F20F76EA66AA68E0800F5CF0CF0EB
:104F90000CC04DF0820E056E080E0A6E820E066E73
:104FA000040E076E010E0B6E4D50106E05EC01F0F5
:104FB000452AD8B4462AD8A4CFD712000000000052
:104FC0000000000000000000000000000000008061
:104FD00080808080808000000000000000000000D1
:104FE0000000000000000000008080808080808041
:104FF00000000000000000000000000000000000B1
:105000000000000000000000000000008000000020
:10501000000000000000000000000080E0F0F8FC4C
:10502000FEFFFFFFFFFFFFFFFFFFFFFFFEFCF8F0AB
:10503000E0000000000000000000000000EF080891
:10504000080808FBF800FCE4040404FC00FCE00091
:105050000000FC00FCE4040404FC00FCE404040480
:10506000FF00000000000000F80C020101C1FFFF7A
:10507000FF1F07030301010303071FFB03030100D5
:1050800000000001033FF8000000000000000000E5
:105090000001010101010101C1C0C1C1C1C1C1C102
:1050A000C0C10101C1C1C1C0C1C1C0C0C0C10001F6
:1050B0000101010101000000000000000F3C3C7CE8
:1050C0007C7FFFFFFFF0E0C0C0E0E0F0F87C3F0F26
:1050D000000000000000000080FC1F000000000035
:1050E000000000000000000000000000FFFF0000C2
:1050F00000000F1FFFFF0000FFFFF0E000000000B6
:10510000FFFF0000000000000000000000000000A1
:1051100000000000000000030F3F7FFFE5C180207A
:1051200000000000008080C06030180E0300000006
:10513000000000000000000000000000000000006F
:105140000303030303030303030300000303030335
:105150000000000003030000000000000000000049
:10516000000000000000000000000000000000003F
:105170000001010101030101010100000000000024
:1051800000000000000000000000000000007CFEA5
:10519000FEFEFEBAD6EED6BAFEFEFEFE7C00000093
:1051A000000000007CFEFEFEFEEEDEBECEF2FAFE49
:1051B000FEFE7C00120092EC24F094988288456AEE
:1051C000466A010E465CD8A0EEEF28F0D8A412EF94
:1051D00029F0F80E455CD8B012EF29F0520E0F6E90
:1051E000260E0E6E45500E24F66E46500F20F76EBA
:1051F000A66AA68E0800F5CF0CF00CC04DF0820E0A
:10520000056E080E0A6E820E066E040E076E010E03
:105210000B6E4D50106E05EC01F0452AD8B4462AAD
:10522000D8A4CFD71200000000000000000000004A
:1052300000000000000000000080808080808080EE
:10524000000000000000000000000000000000005E
:1052500000000080808080808080000000000000CE
:10526000000000000000000000000000000000003E
:1052700000000000000080000000000000000000AE
:10528000000000000080E0F0F8FCFEFFFFFFFFFFE1
:10529000FFFFFFFFFFFFFEFCF8F0E0000000000052
:1052A00000000000000000EF0808080808FBF800F4
:1052B000FCE4040404FC00FCE0000000FC00FCE44E
:1052C000040404FC00FCE4040404FF0000000000EB
:1052D0000000F80C020101C1FFFFFF1F07030301DB
:1052E000010303071FFB030301000080808183BFCC
:1052F000B80000000000000000000001010101C131
:10530000C1C1C1C0C1C1C1C1C10100C1C1C1C1C10F
:10531000C1C0C10100C0C0C1C0C1C1C1C101010043
:105320000000000000000F3C3C7C7C7FFFFFFFF092
:10533000E0C0C0E0E0F0F81CE7FBFC7E1E3F7FF71A
:10534000E3C3837B1B070F1E3EFCF08000000000C0
:10535000000000FFFF000000000F1FFFFF0000FF24
:10536000FFF8F8181818180000FFFFF8F8181818B8
:105370001800000000000000000000000000000015
:1053800000030F3F7FFFE5C1802000001F3F7FFC2F
:10539000E0C0A0B0990B070F9EFCF8F0F87F3F0724
:1053A00000000000000000030303030303030303E2
:1053B00003000003030303000000000000030303D5
:1053C00003000000000000000000000000000000DA
:1053D00000000000000000000000000101010103C6
:1053E000010101000101030303030303030301019E
:1053F00000000000000000007CFEFEFEFEBAD6EEBB
:10540000D6BAFEFEFEFE7C000000000000007CFE1E
:10541000FEFEFEEEDEBECEF2FAFEFEFE7C001200C6
:1054200092EC24F094988288456A466A010E465CA4
:10543000D8A023EF2AF0D8A447EF2AF0F80E455C55
:10544000D8B047EF2AF0540E0F6E900E0E6E4550F6
:105450000E24F66E46500F20F76EA66AA68E080040
:10546000F5CF0CF00CC04DF0820E056E080E0A6EE2
:10547000820E066E040E076E010E0B6E4D50106EFE
:1054800005EC01F0452AD8B4462AD8A4CFD712009B
:10549000000000000000000000000000000000000C
:1054A00000800000404040404040408080000000BC
:1054B00000000000000000000000000000000000EC
:1054C000000080000000000000808000000000005C
:1054D000000000800000000000000000000000004C
:1054E000000000000000000000000000000000A01C
:1054F00008000201010000000000000000000000A0
:10550000000101020C30C00000000000000000009B
:10551000000000000000FFF0F000000000FEF000BE
:10552000FCE4040404FC00FFE4040404FC0004FFA5
:10553000E404000000000000000000000000000083
:10554000000000040000000000020431C020A1E0BF
:1055500021C018020000000080700F000000000051
:1055600000000000000000000000010101C1C1C1F5
:10557000C0C1C1C0C9C9C90909CFC0C1C1C0C0C06B
:10558000C1C0C001010000000000000000000000D8
:105590000000000000000000000002047000000095
:1055A00000163FFB560000000078060100000000D6
:1055B00000000000000000000000000000000000EB
:1055C00000FFFF000000000F1FFFFF0000FFFFF0C3
:1055D000E000000000FFFF000000000000000000ED
:1055E00000000000000000000000000000000000BB
:1055F0000001FEFEFEFEF75752127EFE0100000083
:10560000000000000000000000000000000000009A
:10561000000000000003030303030303030303006C
:105620000003030303000000000303000000000068
:10563000000000000000000000000000000000006A
:105640000000000000000103070F0F0F0F07030108
:10565000000000000000000000000000000000004A
:1056600000007CFEFEFEFEBAD6EED6BAFEFEFEFEC0
:105670007C000000000000007CFEFEFEFEEEDEBEB0
:10568000CEF2FAFEFEFE7C00120092EC24F094981A
:105690008288456A466A010E465CD8A058EF2BF016
:1056A000D8A47CEF2BF0F80E455CD8B07CEF2BF043
:1056B000560E0F6EFA0E0E6E45500E24F66E4650C4
:1056C0000F20F76EA66AA68E0800F5CF0CF00CC06E
:1056D0004DF0820E056E080E0A6E820E066E040EE6
:1056E000076E010E0B6E4D50106E05EC01F0452A51
:1056F000D8B4462AD8A4CFD712000000000000007A
:105700000000000000000000000000800000404099
:105710004040404040808000000000000000000049
:1057200000000000000000000000000080000000F9
:1057300000000080800000000000000000800000E9
:105740000000000000000000000000000000000059
:10575000000000000000000000A00800020101009D
:1057600000000000000000000000000101020C30F9
:10577000C000000000000000000000000000000069
:10578000FFF0F000000000FEF000FCE4040404FC64
:1057900000FFE4040404FC0004FFE4040000000033
:1057A00000000000000000000000000000040000F5
:1057B000000000020431C020A1E021C01802000056
:1057C000000080700F0000000000000000000000DA
:1057D000000000C0C1C1C1C1C1C1C0C1C10009C96F
:1057E000C9C9C9CFC0C1C10000C0C1C0C0C1C1C00A
:1057F000C0000000000000000000000000000000E9
:10580000000000000204700000000096EFF3FA7838
:10581000FCFCDEAE0E0E0E0E1C3C78F8F0C0000054
:1058200000000000000000FFFF000000000F1FFF4D
:10583000FF0000FFFFF8F8181818180000FFFFF825
:10584000F818181818000000000000000000000000
:10585000000000000000000000000001FEFE803F8C
:10586000FFFFF1827EFF03070F1E3C78F0E0C0E0EF
:10587000FFFF1E00000000000000000303030303FD
:1058800003030303030000030303030000000000FD
:1058900000030303030000000000000000000000FC
:1058A00000000000000000000000000000000000F8
:1058B0000103070E0C090B07070E0E0E0C0C0C0E45
:1058C0000F07070301000000000000007CFEFEFE41
:1058D000FEBAD6EED6BAFEFEFEFE7C000000000048
:1058E00000007CFEFEFEFEEEDEBECEF2FAFEFEFE06
:1058F0007C001200436A040E446E97EC24F09498E6
:105900008288456A466A4652D8A4B0EF2CF0A80EA9
:10591000455CD8B0B0EF2CF0590E0F6E620E0E6ED3
:1059200045500E24F66E46500F20F76EA66AA68EDE
:105930000800F5CF0CF00CC04DF0820E056E080E7D
:105940000A6E820E066E040E076E010E0B6E4D502F
:10595000106E05EC01F0452AD8B4462AD8A4D3D756
:105960001200808080808080808080808080808025
:105970008080808080808080808080808080808027
:105980008080808080808080808080808080808017
:105990008080808080808080808080808080808007
:1059A00080808080808080808080808080808080F7
:1059B000808080808080007CFEFEFEFEFE82EAEA1F
:1059C000FAFEFEFEFE7C000000000000007CFEFEF1
:1059D000FEFE82F6EEF682FEFEFEFE7C0000000079
:1059E000000000007CFEFEFEFEAAC692C6AAFEFED5
:1059F000FEFE7C000000000000007CFEFEFEFEC6F5
:105A0000BABABAD6FEFEFEFE7C001200436A040E4D
:105A1000446E97EC24F094988288456A466A465210
:105A2000D8A43CEF2DF0A80E455CD8B03CEF2DF08B
:105A30005A0E0F6E7A0E0E6E45500E24F66E4650BC
:105A40000F20F76EA66AA68E0800F5CF0CF00CC0EA
:105A50004DF0820E056E080E0A6E820E066E040E62
:105A6000076E010E0B6E4D50106E05EC01F0452ACD
:105A7000D8B4462AD8A4D3D71200808080808080F2
:105A80008080808080808080808080808080808016
:105A90008080808080808080808080808080808006
:105AA00080808080808080808080808080808080F6
:105AB00080808080808080808080808080808080E6
:105AC0008080808080808080808080808080007C5A
:105AD000FEFEFEFEBAD6EED6BAFEFEFEFE7C00004C
:105AE00000000000007CFEFEFEFEEECE82CEEEFE4A
:105AF000FEFEFE7C00000000000000007CFEFEC6F2
:105B0000BABAC6FE82EED6BAFEFE7C0000000000E5
:105B100000007CFEFEFEFEEEE682E6EEFEFEFEFEEF
:105B20007C001200436A040E446E97EC24F09498B3
:105B30008288456A466A4652D8A4C8EF2DF0A80E5E
:105B4000455CD8B0C8EF2DF05B0E0F6E920E0E6E56
:105B500045500E24F66E46500F20F76EA66AA68EAC
:105B60000800F5CF0CF00CC04DF0820E056E080E4B
:105B70000A6E820E066E040E076E010E0B6E4D50FD
:105B8000106E05EC01F0452AD8B4462AD8A4D3D724
:105B900012008080808080808080808080808080F3
:105BA00080808080808080808080808080808080F5
:105BB00080808080808080808080808080808080E5
:105BC00080808080808080808080808080808080D5
:105BD00080808080808080808080808080808080C5
:105BE000808080808080007CFEFEFEFEBAD6EED6ED
:105BF000BAFEFEFEFE7C000000000000007CFEFEFF
:105C0000FEFEEEEEEEEEEEFEFEFEFE7C000000007E
:105C1000000000007CFEFEC6BABAC6FE82EED6BA0E
:105C2000FEFE7C000000000000007CFEFEFEFEEE9A
:105C3000EE82EEEEFEFEFEFE7C001200436A040ED3
:105C4000446E97EC24F094988288456A466A4652DE
:105C5000D8A454EF2EF0A80E455CD8B054EF2EF027
:105C60005C0E0F6EAA0E0E6E45500E24F66E465058
:105C70000F20F76EA66AA68E0800F5CF0CF00CC0B8
:105C80004DF0820E056E080E0A6E820E066E040E30
:105C9000076E010E0B6E4D50106E05EC01F0452A9B
:105CA000D8B4462AD8A4D3D71200808080808080C0
:105CB00080808080808080808080808080808080E4
:105CC00080808080808080808080808080808080D4
:105CD00080808080808080808080808080808080C4
:105CE00080808080808080808080808080808080B4
:105CF0008080808080808080808080808080007C28
:105D0000FEFEFEFEBAD6EED6BAFEFEFEFE7C000019
:105D10000000000000000000000000000000000083
:105D20000000000000000000000000000000000073
:105D30000000000000000000000000000000000063
:105D40000000000000000000000000000000000053
:105D5000000012004B0E436E446A97EC24F09498B6
:105D60008288456A466A4652D8A4E0EF2EF0080EB3
:105D7000455CD8B0E0EF2EF05D0E0F6EC20E0E6ED9
:105D800045500E24F66E46500F20F76EA66AA68E7A
:105D90000800F5CF0CF00CC04DF0820E056E080E19
:105DA0000A6E820E066E040E076E010E0B6E4D50CB
:105DB000106E05EC01F0452AD8B4462AD8A4D3D7F2
:105DC00012007F7F3E3E1C1C080812004B0E436EE3
:105DD000446A97EC24F094988288456A466A465251
:105DE000D8A41CEF2FF0080E455CD8B01CEF2FF0A4
:105DF0005E0E0F6E3A0E0E6E45500E24F66E465035
:105E00000F20F76EA66AA68E0800F5CF0CF00CC026
:105E10004DF0820E056E080E0A6E820E066E040E9E
:105E2000076E010E0B6E4D50106E05EC01F0452A09
:105E3000D8B4462AD8A4D3D712007F7F007F7F0032
:105E400000001200436A446A97EC24F0200E4D6E65
:105E5000430E4E6E610E4F6E6C0E506E690E516E9B
:105E6000620E526E720E536E610E546E740E556E4B
:105E7000690E566E6F0E576E6E0E586E200E596E6E
:105E80005A6E5B6A61EC24F0A1DF1200436A010ED6
:105E9000446E97EC24F094988288456A466A010E15
:105EA000465CD8A05CEF2FF0D8A480EF2FF0500E06
:105EB000455CD8B080EF2FF0630E0F6E520E0E6E61
:105EC00045500E24F66E46500F20F76EA66AA68E39
:105ED0000800F5CF0CF00CC04DF0820E056E080ED8
:105EE0000A6E820E066E040E076E010E0B6E4D508A
:105EF000106E05EC01F0452AD8B4462AD8A4CFD7B5
:105F0000960E3BEC01F0436A010E446E97EC24F0D0
:105F100094988288456A466A010E465CD8A099EF3B
:105F20002FF0D8A4BDEF2FF0500E455CD8B0BDEFD8
:105F30002FF0640E0F6EA40E0E6E45500E24F66EFA
:105F400046500F20F76EA66AA68E0800F5CF0CF01B
:105F50000CC04DF0820E056E080E0A6E820E066EA3
:105F6000040E076E010E0B6E4D50106E05EC01F025
:105F7000452AD8B4462AD8A4CFD7FA0E3BEC01F074
:105F8000436A010E446E97EC24F094988288456A27
:105F9000466A010E465CD8A0D6EF2FF0D8A4FAEFDF
:105FA0002FF0500E455CD8B0FAEF2FF0650E0F6E53
:105FB000F60E0E6E45500E24F66E46500F20F76E0C
:105FC000A66AA68E0800F5CF0CF00CC04DF0820E2C
:105FD000056E080E0A6E820E066E040E076E010E26
:105FE0000B6E4D50106E05EC01F0452AD8B4462AD0
:105FF000D8A4CFD7FA0E3BEC01F0436A010E446EF1
:1060000097EC24F094988288456A466A010E465CB3
:10601000D8A013EF30F0D8A437EF30F0500E455C25
:10602000D8B037EF30F0670E0F6E480E0E6E455049
:106030000E24F66E46500F20F76EA66AA68E080054
:10604000F5CF0CF00CC04DF0820E056E080E0A6EF6
:10605000820E066E040E076E010E0B6E4D50106E12
:1060600005EC01F0452AD8B4462AD8A4CFD7960E1D
:106070003BEC01F0436A010E446E97EC24F09498D7
:106080008288456A466A010E465CD8A050EF30F01F
:10609000D8A474EF30F0500E455CD8B074EF30F0F7
:1060A000680E0F6E9A0E0E6E45500E24F66E465018
:1060B0000F20F76EA66AA68E0800F5CF0CF00CC074
:1060C0004DF0820E056E080E0A6E820E066E040EEC
:1060D000076E010E0B6E4D50106E05EC01F0452A57
:1060E000D8B4462AD8A4CFD7960E3BEC01F0436A29
:1060F000010E446E97EC24F094988288456A466AB3
:10610000010E465CD8A08DEF30F0D8A4B1EF30F08E
:10611000500E455CD8B0B1EF30F0690E0F6EEC0E4A
:106120000E6E45500E24F66E46500F20F76EA66A8E
:10613000A68E0800F5CF0CF00CC04DF0820E056E57
:10614000080E0A6E820E066E040E076E010E0B6EAE
:106150004D50106E05EC01F0452AD8B4462AD8A45B
:10616000CFD7960E3BEC01F0436A010E446E97ECDC
:1061700024F094988288456A466A010E465CD8A04D
:10618000CAEF30F0D8A4EEEF30F0500E455CD8B036
:10619000EEEF30F06B0E0F6E3E0E0E6E45500E247D
:1061A000F66E46500F20F76EA66AA68E0800F5CF51
:1061B0000CF00CC04DF0820E056E080E0A6E820EB9
:1061C000066E040E076E010E0B6E4D50106E05EC40
:1061D00001F0452AD8B4462AD8A4CFD7960E3BEC76
:1061E00001F0436A010E446E97EC24F09498828883
:1061F000456A466A010E465CD8A007EF31F0D8A484
:106200002BEF31F0500E455CD8B02BEF31F06C0E17
:106210000F6E900E0E6E45500E24F66E46500F20F7
:10622000F76EA66AA68E0800F5CF0CF00CC04DF0F4
:10623000820E056E080E0A6E820E066E040E076E42
:10624000010E0B6E4D50106E05EC01F0452AD8B4CE
:10625000462AD8A4CFD7960E3BEC01F0436A010E34
:10626000446E97EC24F094988288456A466A010E41
:10627000465CD8A044EF31F0D8A468EF31F0500E5E
:10628000455CD8B068EF31F06D0E0F6EE20E0E6E09
:1062900045500E24F66E46500F20F76EA66AA68E65
:1062A0000800F5CF0CF00CC04DF0820E056E080E04
:1062B0000A6E820E066E040E076E010E0B6E4D50B6
:1062C000106E05EC01F0452AD8B4462AD8A4CFD7E1
:1062D000960E3BEC01F0436A010E446E97EC24F0FD
:1062E00094988288456A466A010E465CD8A081EF80
:1062F00031F0D8A4A5EF31F0500E455CD8B0A5EF31
:1063000031F06F0E0F6E340E0E6E45500E24F66E89
:1063100046500F20F76EA66AA68E0800F5CF0CF047
:106320000CC04DF0820E056E080E0A6E820E066ECF
:10633000040E076E010E0B6E4D50106E05EC01F051
:10634000452AD8B4462AD8A4CFD7960E3BEC01F004
:10635000120000000000000000000000000000002B
:10636000000000000000000000000000000000002D
:1063700000000000E0E0A0A0A0A0A0A0A0A0A0A01D
:10638000A0E0E000000000000000000000000000AD
:1063900000000000000000000000000000000000FD
:1063A00000000000000000000000000000000000ED
:1063B00000000000000000000000000000000000DD
:1063C0000000000000000000001F3F60C0800000CF
:1063D0000080C0603F1F00000000000000000000BF
:1063E00000000000000000000000000000000000AD
:1063F000000000000000000000000000000000009D
:10640000000000000000000000000000000000008C
:1064100000000000000000000000000000F0F88C08
:1064200046A351A851A3468CF8F0000000000000DC
:10643000000000000000000000000000000000005C
:10644000000000000000000000000000000080804C
:10645000808080808080808080808080808080803C
:10646000808080808080808080808080808080802C
:106470008E8F8B8A8B8A8B8A8B8A8B8A8B8F8E806E
:10648000808080808080808080808080808080800C
:1064900080808080808080808080808080808080FC
:1064A00080801200000000000000000000000000DA
:1064B00000000000000000000000000000000000DC
:1064C00000000000000000000000000000000000CC
:1064D00000000000000000000000000000000000BC
:1064E00000000000000000000000000000000000AC
:1064F000000000000000000000000000000000009C
:10650000000000000000000000000000000000008B
:10651000000000000000FE06FEAC5CAC4C8C1830A5
:1065200060C06030180C0C0C0C0CFE06FE00000065
:10653000000000000000000000000000000000005B
:10654000000000000000000000000000000000004B
:10655000000000000000000000000000000000003B
:1065600000000000000000000000FFC0FF6A756A24
:10657000656231180C060C18306060606060FFC006
:10658000FF0000000000000000000000000000000C
:1065900000000000000000000000000000000000FB
:1065A00080808080808080808080808080808080EB
:1065B00080808080808080808080808080808080DB
:1065C00080808080808080808080808080808080CB
:1065D00080808080808080808080808080808080BB
:1065E00080808080808080808080808080808080AB
:1065F0008080808012000000000000000000000089
:10660000000000000000000000000000000000008A
:106610000000000000000000E0E0A0A0A0A0A0A0FA
:10662000A0A0A0A0A0E0E00000000000000000008A
:10663000000000000000000000000000000000005A
:10664000000000000000000000000000000000004A
:10665000000000000000000000000000000000003A
:10666000000000000000000000000000001F3F626A
:10667000C58A15AA158AC5623F1F000000000000E8
:10668000000000000000000000000000000000000A
:1066900000000000000000000000000000000000FA
:1066A00000000000000000000000000000000000EA
:1066B00000000000000000000000000000000000DA
:1066C00000F0F80C060301000103060CF8F00000CE
:1066D00000000000000000000000000000000000BA
:1066E00000000000000000000000000000000000AA
:1066F000000080808080808080808080808080809A
:106700008080808080808080808080808080808089
:10671000808080808E8F8B8A8A8A8A8A8A8A8A8AF7
:106720008B8F8E8080808080808080808080808041
:106730008080808080808080808080808080808059
:106740008080808080801200000000000000000037
:106750000000000000000000000000000000000039
:1067600000000000000000000000E0E0A0A0A0A0E9
:10677000A0A0A0A0A0A0A0E0E000000000000000F9
:106780000000000000000000000000000000000009
:1067900000000000000000000000000000000000F9
:1067A00000000000000000000000000000000000E9
:1067B0000000000000000000000000000000001FBA
:1067C0003F62C58A15AA158AC5623F1F00000000F6
:1067D00000000000000000000000000000000000B9
:1067E00000000000000000000000000000000000A9
:1067F0000000000000000000000000000000000099
:106800000000000000000000000000000000000088
:10681000000000F0F80C060301AA0103060CF8F0D2
:106820000000000000000000000000000000000068
:106830000000000000000000000000000000000058
:106840000000000080808080808080808080808048
:106850008080808080808080808080808080808038
:106860008080808080808E8F8B8A8A8A8A8A8A8ABA
:106870008A8A8B8F8E8080808080808080808080DC
:106880008080808080808080808080808080808008
:1068900080808080808080801200000000000000E6
:1068A00000000000000000000000000000000000E8
:1068B000000000000000000000000000E0E0A0A0D8
:1068C000A0A0A0A0A0A0A0A0A0E0E0000000000068
:1068D00000000000000000000000000000000000B8
:1068E00000000000000000000000000000000000A8
:1068F0000000000000000000000000000000000098
:106900000000000000000000000000000000000087
:10691000001F3F62C58A15AA158AC5623F1F000085
:106920000000000000000000000000000000000067
:106930000000000000000000000000000000000057
:106940000000000000000000000000000000000047
:106950000000000000000000000000000000000037
:106960000000000000F0F80C060301AA0103060C69
:10697000F8F000000000000000000000000000002F
:106980000000000000000000000000000000000007
:1069900000000000000080808080808080808080F7
:1069A00080808080808080808080808080808080E7
:1069B00080808080808080808E8F8B8A8A8A8B8A7C
:1069C0008B8A8A8A8B8F8E80808080808080808076
:1069D00080808080808080808080808080808080B7
:1069E0008080808080808080808012000000000095
:1069F0000000000000000000000000000000000097
:106A00000000000000000000000000000000E0E0C6
:106A1000A0A0A0A0A0A0A0A0A0A0A0E0E0000000D6
:106A20000000000000000000000000000000000066
:106A30000000000000000000000000000000000056
:106A40000000000000000000000000000000000046
:106A50000000000000000000000000000000000036
:106A60000000001F3F60C48A14A8148AC4603F1F3E
:106A70000000000000000000000000000000000016
:106A80000000000000000000000000000000000006
:106A900000000000000000000000000000000000F6
:106AA00000000000000000000000000000000000E6
:106AB00000000000000000F0F80C068301AA01832A
:106AC000060CF8F0000000000000000000000000CC
:106AD00000000000000000000000000000000000B6
:106AE00000000000000000008080808080808080A6
:106AF0008080808080808080808080808080808096
:106B0000808080808080808080808E8F8B8A8B8A3E
:106B10008B8A8B8A8B8A8B8F8E808080808080800E
:106B20008080808080808080808080808080808065
:106B30008080808080808080808080801200000043
:106B40000000000000000000000000000000000045
:106B50000000000000000000000000000000000035
:106B6000E0E0A0A0A0A0A0A0A0A0A0A0A0E0E000C5
:106B70000000000000000000000000000000000015
:106B80000000000000000000000000000000000005
:106B900000000000000000000000000000000000F5
:106BA00000000000000000000000000000000000E5
:106BB00000000000001F3F60C48810A81088C46057
:106BC0003F1F000000000000000000000000000067
:106BD00000000000000000000000000000000000B5
:106BE00000000000000000000000000000000000A5
:106BF0000000000000000000000000000000000095
:106C0000000000000000000000F0F80C068341AA1C
:106C10004183060CF8F000000000000000000000B6
:106C20000000000000000000000000000000000064
:106C30000000000000000000000080808080808054
:106C40008080808080808080808080808080808044
:106C50008080808080808080808080808E8F8B8A02
:106C60008B8A8B8A8B8A8B8A8B8F8E8080808080A8
:106C70008080808080808080808080808080808014
:106C800080808080808080808080808080801200F2
:106C900000000000000000000000000000000000F4
:106CA00000000000000000000000000000000000E4
:106CB0000000E0E0A0A0A0A0A0A0A0A0A0A0A0E054
:106CC000E0000000000000000000000000000000E4
:106CD00000000000000000000000000000000000B4
:106CE00000000000000000000000000000000000A4
:106CF0000000000000000000000000000000000094
:106D0000000000000000001F3F60C08810A810882D
:106D1000C0603F1F000000000000000000000000F5
:106D20000000000000000000000000000000000063
:106D30000000000000000000000000000000000053
:106D40000000000000000000000000000000000043
:106D50000000000000000000000000F0F88C4683F6
:106D600041AA4183468CF8F00000000000000000BA
:106D70000000000000000000000000000000000013
:106D80000000000000000000000000008080808003
:106D900080808080808080808080808080808080F3
:106DA00080808080808080808080808080808E8FC6
:106DB0008B8A8B8A8B8A8B8A8B8A8B8F8E80808042
:106DC00080808080808080808080808080808080C3
:106DD00080808080808080808080808080808080B3
:106DE0001200000000000000000000000000000091
:106DF0000000000000000000000000000000000093
:106E000000000000E0E0A0A0A0A0A0A0A0A0A0A082
:106E1000A0E0E00000000000000000000000000012
:106E20000000000000000000000000000000000062
:106E30000000000000000000000000000000000052
:106E40000000000000000000000000000000000042
:106E50000000000000000000001F3F60C08010A084
:106E60001080C0603F1F0000000000000000000014
:106E70000000000000000000000000000000000012
:106E80000000000000000000000000000000000002
:106E900000000000000000000000000000000000F2
:106EA00000000000000000000000000000F0F88C6E
:106EB00046A351AA51A3468CF8F000000000000040
:106EC00000000000000000000000000000000000C2
:106ED00000000000000000000000000000008080B2
:106EE00080808080808080808080808080808080A2
:106EF0008080808080808080808080808080808092
:106F00008E8F8B8A8B8A8B8A8B8A8B8A8B8F8E80D3
:106F10008080808080808080808080808080808071
:106F20008080808080808080808080808080808061
:106F3000808012000000000000000000000000003F
:106F40000000000000000000000000000000000041
:106F5000000000000000E0E0A0A0A0A0A0A0A0A071
:106F6000A0A0A0E0E0000000000000000000000081
:106F70000000000000000000000000000000000011
:106F80000000000000000000000000000000000001
:106F900000000000000000000000000000000000F1
:106FA00000000000000000000000001F3F60C080E3
:106FB00000000080C0603F1F0000000000000000D3
:106FC00000000000000000000000000000000000C1
:106FD00000000000000000000000000000000000B1
:106FE00000000000000000000000000000000000A1
:106FF000000000000000000000000000000000F0A1
:10700000F88C46A351AA51A3468CF8F0000000006A
:107010000000000000000000000000000000000070
:107020000000000000000000000000000000000060
:107030008080808080808080808080808080808050
:107040008080808080808080808080808080808040
:1070500080808E8F8B8A8B8A8B8A8B8A8B8A8B8F90
:107060008E80808080808080808080808080808012
:107070008080808080808080808080808080808010
:1070800080808080120092EC24F094988288456A77
:10709000466A010E465CD8A056EF38F0D8A47AEFC5
:1070A00038F0F80E455CD8B07AEF38F0700E0F6EFD
:1070B000F60E0E6E45500E24F66E46500F20F76EFB
:1070C000A66AA68E0800F5CF0CF00CC04DF0820E1B
:1070D000056E080E0A6E820E066E040E076E010E15
:1070E0000B6E4D50106E05EC01F0452AD8B4462ABF
:1070F000D8A4CFD712000000000000000404FCE474
:107100000400FC1010F000F4C400705050D00000D7
:107110000000F01010F000F0101000F01010F0005F
:1071200000F400F050507000F01010100010F8D073
:1071300000000000F00000F0C000F000D05050F05F
:1071400000705050D000000000000080808080005F
:10715000808081018080818000818081810081C167
:1071600081018080808007818181E001000000E151
:10717000818181008407008101010100E1E1212179
:10718000E000016120202020E10101010101010056
:10719000E1E1212120E1016121202020E000000F18
:1071A000080808000F0000000F0A0A0B000E0A0A68
:1071B0000F00000F0E000F0A0A0B000F08080F0047
:1071C0000000000F08080F002F28283F00000000D3
:1071D0000F0F0101010F000F090909090900010141
:1071E000010100000F0F0808080F000F0909090925
:1071F00009000000000000000000000001017F798C
:1072000001007F04047C007C54545C000000007C7E
:1072100054545C000808080800007C04047C7404D2
:107220007C007454547C007D71007F780000000065
:10723000047F75017C44447C007C0404040000004D
:107240000000000000000000E02020E000E000005E
:10725000E000E0A0A0E000E0A0A0A00020F0A000DE
:10726000E88800E02020E000E02020E000E0A0A08E
:10727000A000000000C0F8484848E800000000E016
:107280002020E00020F8A80820F8A808E0A0A0E04E
:1072900000E0202000E0A0A0A00000000302020FF8
:1072A00000030202030003020202000202020300C2
:1072B00000030300030300030202030003000003B2
:1072C00000020202030000000003030202020300A6
:1072D0000000000302020300000303000003030098
:1072E0000302020200030000000202020300120077
:1072F00092EC24F094988288456A466A010E465CB6
:10730000D8A08BEF39F0D8A4AFEF39F0F80E455C78
:10731000D8B0AFEF39F0730E0F6E600E0E6E4550A1
:107320000E24F66E46500F20F76EA66AA68E080051
:10733000F5CF0CF00CC04DF0820E056E080E0A6EF3
:10734000820E066E040E076E010E0B6E4D50106E0F
:1073500005EC01F0452AD8B4462AD8A4CFD71200AC
:10736000000000000000000000000000000000001D
:10737000000000000000000000000000000000000D
:1073800000000000000000000000000000000000FD
:1073900000000000000000000000000000000000ED
:1073A00000000000000000000000000000000000DD
:1073B00000000000000000000000000000000000CD
:1073C00000000000000000000000000000000000BD
:1073D00000000000000000000000000000000000AD
:1073E000000000000000000000000000000000009D
:1073F000000000000000000000000000000000008D
:107400000000000000000000F84848C830001008E4
:10741000C83000204080402000204080402000F8FC
:10742000080808F0001008C83000E010C828C84854
:1074300010E000C02020E000E02020C02020C0009C
:1074400080A0A0E000E800F8000000C0202040007C
:10745000C02020C000E02020C02020C00300000089
:107460000300020302020002010001020002010007
:1074700001020003020202010002030202000304EF
:107480000B0A0B0A090400010A0A070003000003A3
:1074900000000300030202030003000300020001D6
:1074A00002020100010202010003000003000003C8
:1074B00000000000000000000000000000000000CC
:1074C00000000000000000000000000000000000BC
:1074D00000000000000000000000000000000000AC
:1074E000000000000000000000000000000000009C
:1074F000000000000000000000000000000000008C
:10750000000000000000000000000000000000007B
:10751000000000000000000000000000000000006B
:10752000000000000000000000000000000000005B
:10753000000000000000000000000000000000004B
:10754000000000000000000000000000000000003B
:107550000000000000000000120092EC24F094985B
:107560008288456A466A010E465CD8A0C0EF3AF0B0
:10757000D8A4E4EF3AF0F80E455CD8B0E4EF3AF066
:10758000750E0F6ECA0E0E6E45500E24F66E4650E6
:107590000F20F76EA66AA68E0800F5CF0CF00CC07F
:1075A0004DF0820E056E080E0A6E820E066E040EF7
:1075B000076E010E0B6E4D50106E05EC01F0452A62
:1075C000D8B4462AD8A4CFD712000000000000008B
:1075D000000000E8880020F8A808000000E0000093
:1075E000E000E02020E000E00000E000000000F803
:1075F000C000E88800F88080E000E0A0A0E000E0A3
:107600002020F80000000020F0A000F82020E0007A
:10761000E0A0A0E00000000000000000000000006A
:10762000000000000000000303000003030000004E
:10763000000B0A0A0F4003020203000302020300C8
:1076400000008003030003030003000003000302A3
:107650000202000302C20300000000000303000353
:10766000000003000302020200000000000000000E
:10767000000000000000000000007F11111F001F2B
:107680000101001F11111F00407F001F1515170079
:107690001F11111100011F1D000000001D15151FF5
:1076A000001F01011F001F11111F000000005F508B
:1076B000507F001F11111F001F10101F000000003D
:1076C0000000000000000000F88080F8E080F80072
:1076D000E8A8A8F800F80808F80008FCE80000008E
:1076E0000008FCE800F88888F800000000FE0808A0
:1076F000F800F8A8A8B800FEF000F88888F80000A4
:10770000000008FCE800FE0808F800F8A8A8B80087
:10771000FAE200F80808080000000000000000007D
:107720000000000000000000C04040F000C04040E9
:10773000C000C0C000C000C04040C000F08000C019
:107740004040C000C04040C000C04040C04043C0B6
:1077500000C04040C000C04040C00040E0400000C9
:107760000000000000000000000000000000000019
:1077700000000000000000000000000007040407F3
:1077800000070505050001070407000705050500BA
:1077900007070007040407001F0404070007000090
:1077A00007070007000705050500070000070000A0
:1077B00007070000000000000000000000000000BB
:1077C0000000120092EC24F094988288456A466A80
:1077D000010E465CD8A0F5EF3BF0D8A419EF3CF0C1
:1077E000F80E455CD8B019EF3CF0780E0F6E340EF1
:1077F0000E6E45500E24F66E46500F20F76EA66AA8
:10780000A68E0800F5CF0CF00CC04DF0820E056E70
:10781000080E0A6E820E066E040E076E010E0B6EC7
:107820004D50106E05EC01F0452AD8B4462AD8A474
:10783000CFD7120000000000000000000000000090
:107840000000000000000000000000000000000038
:107850000000001CFC6018FC60380CE0FC1CE8FC1C
:107860001CE8FC1C00C0E4B49C8C04000000000078
:107870000000000000000000000000000000000008
:107880000000000000000000000000000088C86840
:10789000381800E0F058C89800607858D898007000
:1078A000F888F8F0001008C8F8B000E0F058C89860
:1078B000001008C8F8B000607858D898002030F060
:1078C000F818001898D838180070F888F8F0008078
:1078D0004020F0F808101888F8700000000000063A
:1078E000070504040400000307040703000604045A
:1078F000070300060406030102060404070300034D
:107900000704070302060404070300060404070330
:10791000000006070100000607010000000604063B
:107920000301010101070701000607050404000027
:107930000000000000000000000000000000000047
:1079400000000000000000000000000000000070C7
:10795000F08060F080E03080F070A0F070A0F070F7
:107960000080F07020100000000000000000000007
:107970000000000000000000000000000000000007
:10798000000000000000000080E0602020E0C00057
:1079900080C0C0E06000000080C0E020C0E020E0C7
:1079A000C000C0E023E1C00381C020E3C30083C363
:1079B000C0E36300000383C0E020000080C0E0203B
:1079C00080C0C0E06000406020E0C000406020E077
:1079D000C00080C020E0C000000000181F070206A1
:1079E0001F19000000181F07000406051C1F0700D0
:1079F00019131A0F070019131A0F07000F1F100F82
:107A0000070000181F07000406051C1F07040605D1
:107A10001C1F070000181F070000181C1613110078
:107A2000181C161311000F1F100F0700120092EC04
:107A300024F094988288456A466A010E465CD8A074
:107A40002AEF3DF0D8A44EEF3DF0F80E455CD8B0DB
:107A50004EEF3DF07A0E0F6E9E0E0E6E45500E24C8
:107A6000F66E46500F20F76EA66AA68E0800F5CF78
:107A70000CF00CC04DF0820E056E080E0A6E820EE0
:107A8000066E040E076E010E0B6E4D50106E05EC67
:107A900001F0452AD8B4462AD8A4CFD71200000056
:107AA000000008484848F8002020E0A000E020201E
:107AB000E0002020E0A020000000E02020E000E026
:107AC0002020E000E02020E000E0A0A0E000E08036
:107AD00080E0002020E0A020000000F82828E80036
:107AE000E080808000E0800080E020E00000000076
:107AF0000000000000000202020203000000030375
:107B00000003020203000000030300000000030062
:107B10000003000F02020300030202C3C04342C27B
:107B20000200C340404340C000030300000000C304
:107B3000C2424340C302C243404343C00303000365
:107B400000000000000000000000000000001F1105
:107B50001111001F11111F001115151B005F51514C
:107B60007F001D15151F001F04041F000000001FCB
:107B70001F0202031E001E12121212130002020242
:107B80000200001F1F1010101F001E1212121213ED
:107B900000000000000000000000F0FE1212FE00D5
:107BA000F88888F800F88888F800F8A8A8B800F8DD
:107BB000888888000000F88888F800E0F808F80055
:107BC000E03828F8000000F8A8A8D800F88888F85D
:107BD00000F80808F800F88888F800F88888F800A5
:107BE000F888888800F88888F800F8A8A8D80000E5
:107BF00000000000020202C30003C000000000C039
:107C00004040C000C04040C000C04242C203C0402B
:107C100040C00000C040C000C04040C00000C000E4
:107C2000C000C00000C04040C000C30000C000C091
:107C30000000C000C01010C00000000000000000E4
:107C4000000000000000000000000007040407001E
:107C500000000007000007001F04040700070505D7
:107C600005001714141F0007070007000704040786
:107C700000070101070101070007050505000701CD
:107C800001070007040407000704040700000000C0
:107C9000000000000000120092EC24F0949882880A
:107CA000456A466A010E465CD8A05FEF3EF0D8A454
:107CB00083EF3EF0F80E455CD8B083EF3EF07D0ECA
:107CC0000F6E080E0E6E45500E24F66E46500F20B5
:107CD000F76EA66AA68E0800F5CF0CF00CC04DF02A
:107CE000820E056E080E0A6E820E066E040E076E78
:107CF000010E0B6E4D50106E05EC01F0452AD8B404
:107D0000462AD8A4CFD7120000000000E0A0A0E0CF
:107D100000E02020200080E020E000E00000E00003
:107D2000000000E02020E000E02020E000E0202033
:107D3000E000E0A0A0E000E08080E0002020E0A0E3
:107D400020000000F848484878C000A0A0A0E0004B
:107D5000E060C0C060E00000000000000000000023
:107D600003020202000302020200030300030003F5
:107D70000202030000000003000003000F020203E0
:107D800000030202030003020202000300000300DA
:107D900000000303000000000302020202C340438C
:107DA00042C20300030000000003000000000000C6
:107DB000000000001F01011F001F11111F001F0400
:107DC000041F007F11111F001D15151F001F151521
:107DD0001F001F10101F001C1F011F001F11111179
:107DE000001C07051F000000001F10101F000000EE
:107DF000001F121212131E001F14141C001F1C005F
:107E00000000000000D82020D800F88888F800087A
:107E100008F8E800F88080F8000808F8E800F8A8FA
:107E2000A8B800000000F80808F800F88888F800F2
:107E3000F818303018F800F88888F800382020F852
:107E400000F8A0A0E000000000F8A8A8B800F8081A
:107E50000800F88888F8000000000000000000001A
:107E600000000000000000000000000000C04040D2
:107E7000C000404040C000404040C000C04040C042
:107E800000C00000C0004040C04000C00000C00072
:107E9000C000C04040C00000000000000000000022
:107EA00000000000000000000000000000000000D2
:107EB00000000000000000000000000000000000C2
:107EC000001F040407000705050700040505060058
:107ED000070505070007040407000000070700075F
:107EE0000404070007010704040700000000000065
:107EF0000000000000000000000000000000000082
:047F00001200FFD795
:020000040030CA
:0E000000FFF2E2EEFFFDBBFFFFFFFFFFFFFF81
:00000001FF
